:020000040000FA
:04080000EDEF0BF01D
:1008100003B276EF05F0F2B494EF05F09EB09CEFD2
:1008200005F09EB2A4EF05F0F2A81AEF04F0F2B2C0
:1008300025EF04F0F2A620EF04F0F2B022EF04F06E
:100840009CEF0BF0F296F290FF00CD90F2929EA0FA
:100850002FEF04F00101533F2FEF04F0542BAEC1F2
:10086000B2F1AFC1B3F1B0C1B4F1B1C1B5F1AAC138
:10087000AEF1ABC1AFF1ACC1B0F1ADC1B1F1A6C148
:10088000AAF1A7C1ABF1A8C1ACF1A9C1ADF1A2C158
:10089000A6F1A3C1A7F1A4C1A8F1A5C1A9F19EC168
:1008A000A2F19FC1A3F1A0C1A4F1A1C1A5F19AC178
:1008B0009EF19BC19FF19CC1A0F19DC1A1F196C188
:1008C0009AF197C19BF198C19CF199C19DF1CECF4E
:1008D00096F1CFCF97F153C198F154C199F1CF6AF6
:1008E000CE6A0101536B546B9E90CD800FBC0F8E6E
:1008F0000FBA7EEF04F00F8A9CEF0BF00F8C0FBE47
:10090000BAEF04F096C19AF197C19BF198C19CF19E
:1009100099C19DF19AC19EF19BC19FF19CC1A0F12B
:100920009DC1A1F19EC1A2F19FC1A3F1A0C1A4F1FB
:10093000A1C1A5F1A2C1A6F1A3C1A7F1A4C1A8F1CB
:10094000A5C1A9F1A6C1AAF1A7C1ABF1A8C1ACF19B
:10095000A9C1ADF1AAC1AEF1ABC1AFF1ACC1B0F16B
:10096000ADC1B1F1AEC1B2F1AFC1B3F1B0C1B4F13B
:10097000B1C1B5F101015E6B5F6B606B616B96514C
:100980005E2797515F2398516023995161239A51B3
:100990005E279B515F239C5160239D5161239E5193
:1009A0005E279F515F23A0516023A1516123A25173
:1009B0005E27A3515F23A4516023A5516123A65153
:1009C0005E27A7515F23A8516023A9516123AA5133
:1009D0005E27AB515F23AC516023AD516123AE5113
:1009E0005E27AF515F23B0516023B1516123B251F3
:1009F0005E27B3515F23B4516023B5516123D89072
:100A00000101613360335F335E33D890010161339C
:100A100060335F335E33D8900101613360335F33FD
:100A20005E3300C10CF101C10DF102C10EF103C131
:100A30000FF104C110F105C111F106C112F107C196
:100A400013F108C114F109C115F10AC116F10BC166
:100A500017F134C135F111B839EF05F00101620E1B
:100A6000046F010E056F000E066F000E076F42EF58
:100A700005F00101A70E046F020E056F000E066F50
:100A8000000E076F5EC100F15FC101F160C102F1AC
:100A900061C103F15DEC33F003BF04D018BE02D096
:100AA00018A0108C11A05AEF05F010BA5AEF05F0FB
:100AB0000F80108A0CC100F10DC101F10EC102F1CD
:100AC0000FC103F110C104F111C105F112C106F10A
:100AD00013C107F114C108F115C109F116C10AF1DA
:100AE00017C10BF135C134F19CEF0BF00392ABB29F
:100AF000AB98AB88030103EE00F080517F0BE92631
:100B000004C0EFFF802B8151805D700BD8A48B82D5
:100B100000008051815D700BD8A48B9281518019A7
:100B2000D8B407909CEF0BF0F2940101453F9CEF85
:100B30000BF0462B9CEF0BF09E900101533F9CEF76
:100B40000BF0542B9CEF0BF09E9211B871EF08F054
:100B5000040062A1ACEF05F08BB4B6EF05F010AC69
:100B6000B6EF05F08B84109CB7EF05F08B9407B4BB
:100B700009EF06F007B009EF06F01EC620F61FC603
:100B800021F61CC61EF61DC61FF61AC61CF61BC68D
:100B90001DF606C608F607C609F604C606F605C61B
:100BA00007F602C604F603C605F626C628F627C6CB
:100BB00029F624C626F625C627F622C624F623C61D
:100BC00025F60EC610F60FC611F60CC60EF60DC6AB
:100BD0000FF60AC60CF60BC60DF62EC630F62FC65B
:100BE00031F62CC62EF62DC62FF62AC62CF62BC6AD
:100BF0002DF616C618F617C619F614C616F615C63B
:100C000017F612C614F613C615F63EEC35F0ECECEA
:100C100034F0077C07AC24EF06F0C274C2B41EEFB8
:100C200006F0C3CFB3F5C4CFB4F50501D890B43303
:100C3000B333D890B433B33325EF06F0C3CF55F1B7
:100C4000C4CF56F125EF06F0C28207B492EF06F04A
:100C500047C14BF148C14CF149C14DF14AC14EF178
:100C60005EC162F15FC163F160C164F161C165F1B0
:100C700096C1B6F197C1B7F198C1B8F199C1B9F170
:100C80009AC1BAF19BC1BBF19CC1BCF19DC1BDF140
:100C90009EC1BEF19FC1BFF1A0C1C0F1A1C1C1F110
:100CA000A2C1C2F1A3C1C3F1A4C1C4F1A5C1C5F1E0
:100CB000A6C1C6F1A7C1C7F1A8C1C8F1A9C1C9F1B0
:100CC000AAC1CAF1ABC1CBF1ACC1CCF1ADC1CDF180
:100CD000AEC1CEF1AFC1CFF1B0C1D0F1B1C1D1F150
:100CE000B2C1D2F1B3C1D3F1B4C1D4F1B5C1D5F120
:100CF000B3C5B5F5B4C5B6F5B5C5B7F5B6C5B8F560
:100D0000010155515B2756515C23E86A5D230E2E85
:100D100092EF06F05CC157F15DC158F15B6B5C6B03
:100D20005D6B078E0201002F9CEF0BF03C0E006FF5
:100D30001950E00BE00AE866128816AE108E00C16A
:100D40000CF101C10DF102C10EF103C10FF104C19B
:100D500010F105C111F106C112F107C113F108C16B
:100D600014F109C115F10AC116F10BC117F134C113
:100D700035F105012F51000AD8B46AEF07F00501DB
:100D80002F51010AD8B4F4EF06F005012F51020AE1
:100D9000D8B435EF07F005012F51030AD8B435EF69
:100DA00007F005012F51040AD8B435EF07F005010B
:100DB0002F51050AD8B435EF07F005012F51060A67
:100DC000D8B435EF07F005012F51070AD8B435EF35
:100DD00007F005012F51320AD8B4F2EF06F02F6B5D
:100DE0006AEF07F06AEF07F005015367FFEF06F0BF
:100DF0005467FFEF06F05567FFEF06F0566703EF05
:100E000007F06AEF07F057C500F158C501F159C561
:100E100002F15AC503F10101010E046F000E056FC6
:100E2000000E066F000E076F5DEC33F000C157F542
:100E300001C158F502C159F503C15AF5006728EF01
:100E400007F0016728EF07F0026728EF07F0036754
:100E50006AEF07F053C557F554C558F555C559F510
:100E600056C55AF50F886AEF07F0050130673BEF6A
:100E700007F06AEF07F00FBE50EF07F010A055EF34
:100E800007F0010147674CEF07F048674CEF07F0A8
:100E900049674CEF07F04A6750EF07F055EF07F04E
:100EA00007AE55EF07F067EF07F00501312F6AEF46
:100EB00007F03C0E316F302F6AEF07F00101000E92
:100EC000626FE00E636FA50E646F010E656F050122
:100ED000306B0F880501626B33B770EF07F06281EA
:100EE0000CC100F10DC101F10EC102F10FC103F1FE
:100EF00010C104F111C105F112C106F113C107F1CE
:100F000014C108F115C109F116C10AF117C10BF19D
:100F100035C134F100C10CF101C10DF102C10EF176
:100F200003C10FF104C110F105C111F106C112F1A5
:100F300007C113F108C114F109C115F10AC116F175
:100F40000BC117F134C135F101018A67AFEF07F02A
:100F50008B67AFEF07F08C67AFEF07F08D67B3EFEC
:100F600007F0E3EF07F08EC100F18FC101F190C1EE
:100F700002F191C103F10101010E046F000E056F32
:100F8000000E066F000E076F5DEC33F000C18EF1AE
:100F900001C18FF102C190F103C191F10067D8EF57
:100FA00007F00167D8EF07F00267D8EF07F0036793
:100FB000E3EF07F08AC18EF18BC18FF18CC190F104
:100FC0008DC191F10F80D57ED5BE6DD0D6CF47F1C2
:100FD000D7CF48F145C149F1E86AE8CF4AF118BED8
:100FE00002D018A0108C109047C100F148C101F147
:100FF00049C102F14AC103F101010A0E046F000E5A
:10100000056F000E066F000E076F5DEC33F003AF47
:101010001080010154A719EF08F00F9A0F9C0F9E42
:101020000101000E5E6F600E5F6F3D0E606F080E77
:10103000616F010147BF29EF08F0486729EF08F009
:10104000496729EF08F04A6729EF08F0F2884EEF68
:1010500008F0F2985E6B5F6B606B616B966B976BE1
:10106000986B996B9A6B9B6B9C6B9D6B9E6B9F6B4C
:10107000A06BA16BA26BA36BA46BA56BA66BA76BFC
:10108000A86BA96BAA6BAB6BAC6BAD6BAE6BAF6BAC
:10109000B06BB16BB26BB36BB46BB56BD76AD66A1E
:1010A0000101456B466B0CC100F10DC101F10EC190
:1010B00002F10FC103F110C104F111C105F112C118
:1010C00006F113C107F114C108F115C109F116C1E8
:1010D0000AF117C10BF135C134F19CEF0BF09CEF15
:1010E0000BF00201002FB3EF0AF0D59ED6CF47F1E7
:1010F000D7CF48F145C149F1E86AE8CF4AF1D76A4C
:10110000D66A0101456B466BD58E1950E00BE00A9B
:10111000E866128817AE108E16AE1B8C00C10CF15B
:1011200001C10DF102C10EF103C10FF104C110F1B3
:1011300005C111F106C112F107C113F108C114F183
:1011400009C115F10AC116F10BC117F134C135F10E
:101150000FA0109A11B8B8EF08F00101620E046FE9
:10116000010E056F000E066F000E076FC1EF08F04D
:101170000101A70E046F020E056F000E066F000E30
:10118000076F47C100F148C101F149C102F14AC1ED
:1011900003F15DEC33F003BFD4EF08F018BE02D0CA
:1011A00018A0108C11B00F800CC100F10DC101F11D
:1011B0000EC102F10FC103F110C104F111C105F11B
:1011C00012C106F113C107F114C108F115C109F1EB
:1011D00016C10AF117C10BF135C134F102013C0E01
:1011E000006F00C10CF101C10DF102C10EF103C18C
:1011F0000FF104C110F105C111F106C112F107C1CF
:1012000013F108C114F109C115F10AC116F10BC19E
:1012100017F134C135F105012F51000AD8B4BCEFE4
:1012200009F005012F51010AD8B446EF09F0050174
:101230002F51020AD8B487EF09F005012F51030A94
:10124000D8B487EF09F005012F51040AD8B487EF0D
:1012500009F005012F51050AD8B487EF09F00501FF
:101260002F51060AD8B487EF09F005012F51070A5C
:10127000D8B487EF09F005012F51320AD8B444EFF2
:1012800009F02F6BBCEF09F0BCEF09F005015367C3
:1012900051EF09F0546751EF09F0556751EF09F02C
:1012A000566755EF09F0BCEF09F057C500F158C576
:1012B00001F159C502F15AC503F10101010E046F94
:1012C000000E056F000E066F000E076F5DEC33F029
:1012D00000C157F501C158F502C159F503C15AF5CE
:1012E00000677AEF09F001677AEF09F002677AEF99
:1012F00009F00367BCEF09F053C557F554C558F51D
:1013000055C559F556C55AF50F88BCEF09F00501CA
:1013100030678DEF09F0BCEF09F00FBEA2EF09F0C6
:1013200010A0A7EF09F0010147679EEF09F0486799
:101330009EEF09F049679EEF09F04A67A2EF09F0B6
:10134000A7EF09F007AEA7EF09F0B9EF09F0050123
:10135000312FBCEF09F03C0E316F302FBCEF09F09C
:101360000101000E626FE00E636FA50E646F010E47
:10137000656F0501306B0F880501626B33B7C2EFF3
:1013800009F062810CC100F10DC101F10EC102F141
:101390000FC103F110C104F111C105F112C106F131
:1013A00013C107F114C108F115C109F116C10AF101
:1013B00017C10BF135C134F100C10CF101C10DF1C0
:1013C00002C10EF103C10FF104C110F105C111F109
:1013D00006C112F107C113F108C114F109C115F1D9
:1013E0000AC116F10BC117F134C135F101018A6749
:1013F00001EF0AF08B6701EF0AF08C6701EF0AF04A
:101400008D6705EF0AF035EF0AF08EC100F18FC14C
:1014100001F190C102F191C103F10101010E046FCC
:10142000000E056F000E066F000E076F5DEC33F0C7
:1014300000C18EF101C18FF102C190F103C191F1A0
:1014400000672AEF0AF001672AEF0AF002672AEF25
:101450000AF0036735EF0AF08AC18EF18BC18FF174
:101460008CC190F18DC191F10F80109047C100F1B6
:1014700048C101F149C102F14AC103F101010A0E5B
:10148000046F000E056F000E066F000E076F5DEC17
:1014900033F003AF1080010154A75BEF0AF00F9AFD
:1014A0000F9C0F9E0101000E5E6F600E5F6F3D0E80
:1014B000606F080E616F47C100F148C101F149C179
:1014C00002F14AC103F10101140E046F050E056F0C
:1014D000000E066F000E076F5DEC33F003AF74EF84
:1014E0000AF0F28899EF0AF0F2985E6B5F6B606B1E
:1014F000616B966B976B986B996B9A6B9B6B9C6B04
:101500009D6B9E6B9F6BA06BA16BA26BA36BA46B7F
:10151000A56BA66BA76BA86BA96BAA6BAB6BAC6B2F
:10152000AD6BAE6BAF6BB06BB16BB26BB36BB46BDF
:10153000B56B0CC100F10DC101F10EC102F10FC17B
:1015400003F110C104F111C105F112C106F113C17B
:1015500007F114C108F115C109F116C10AF117C14B
:101560000BF135C134F104008BB4BEEF0AF010ACBE
:10157000BEEF0AF08B84109CBFEF0AF08B9407B487
:1015800011EF0BF007B011EF0BF01EC620F61FC6CF
:1015900021F61CC61EF61DC61FF61AC61CF61BC673
:1015A0001DF606C608F607C609F604C606F605C601
:1015B00007F602C604F603C605F626C628F627C6B1
:1015C00029F624C626F625C627F622C624F623C603
:1015D00025F60EC610F60FC611F60CC60EF60DC691
:1015E0000FF60AC60CF60BC60DF62EC630F62FC641
:1015F00031F62CC62EF62DC62FF62AC62CF62BC693
:101600002DF616C618F617C619F614C616F615C620
:1016100017F612C614F613C615F63EEC35F0ECECD0
:1016200034F0077C07AC2CEF0BF0C274C2B426EF89
:101630000BF0C3CFB3F5C4CFB4F50501D890B433E4
:10164000B333D890B433B3332DEF0BF0C3CF55F190
:10165000C4CF56F12DEF0BF0C28207B49AEF0BF016
:1016600047C14BF148C14CF149C14DF14AC14EF15E
:101670005EC162F15FC163F160C164F161C165F196
:1016800096C1B6F197C1B7F198C1B8F199C1B9F156
:101690009AC1BAF19BC1BBF19CC1BCF19DC1BDF126
:1016A0009EC1BEF19FC1BFF1A0C1C0F1A1C1C1F1F6
:1016B000A2C1C2F1A3C1C3F1A4C1C4F1A5C1C5F1C6
:1016C000A6C1C6F1A7C1C7F1A8C1C8F1A9C1C9F196
:1016D000AAC1CAF1ABC1CBF1ACC1CCF1ADC1CDF166
:1016E000AEC1CEF1AFC1CFF1B0C1D0F1B1C1D1F136
:1016F000B2C1D2F1B3C1D3F1B4C1D4F1B5C1D5F106
:10170000B3C5B5F5B4C5B6F5B5C5B7F5B6C5B8F545
:10171000010155515B2756515C23E86A5D230E2E6B
:101720009AEF0BF05CC157F15DC158F15B6B5C6BDC
:101730005D6B078E9CEF0BF002C0E0FF005001C014
:10174000D8FF1000A6B2A2EF0BF00CC0A9FF0BC08F
:10175000A8FFA69EA69CA684F29E550EA76EAA0E72
:10176000A76EA682F28EA694A6B2B4EF0BF00C2A56
:101770001200A96EA69EA69CA680A8500C2A120054
:1017800004012C0E826F31EC0FF058EC34F00C5049
:10179000B9EC0BF0E8CF00F10C50B9EC0BF0E8CF4E
:1017A00001F101AFD9EF0BF00101FF0E026FFF0E47
:1017B000036FFBEC33F02967E5EF0BF00401200E1B
:1017C000826F31EC0FF0EAEF0BF004012D0E826F07
:1017D00031EC0FF025EC32F01200076A0F6A106A44
:1017E000116A126A0F010D0EC16E860EC06E030ED5
:1017F000C26E0F01680E896E130E926E080E8A6E0D
:101800008A6AF30E936E8B6A900E946EC80EB9ECD2
:101810000BF0E8CFE8FF1098E8A0108810A805D0DA
:101820000E0E216E8E0E226E04D00F0E216E8F0EC4
:10183000226EF6EC35F0F18EF19EFC0EB9EC0BF059
:10184000E8CF0BF00BA011800BA211820BA4118426
:101850000BA81188C90EB9EC0BF0E8CF16F0CA0E30
:10186000B9EC0BF0E8CF17F0CB0EB9EC0BF0E8CFEA
:1018700018F0CC0EB9EC0BF0E8CF19F01B6A1C6A1B
:101880000E6A01015B6B5C6B5D6B576B586BF29A78
:101890000101476B486B496B4A6B4B6B4C6B4D6B53
:1018A0004E6B4F6B506B516B526B456B466BD76AEF
:1018B000D66A0F01280ED56EF28A9D90B00ECD6EBD
:1018C00001015E6B5F6B606B616B626B636B646B82
:1018D000656B666B676B686B696B536B546BCF6A38
:1018E000CE6A0F9A0F9C0F9E9D80760ECA6E9D82C7
:1018F00002013C0E006FCC6A160EB9EC0BF0E8CF7B
:1019000000F1170EB9EC0BF0E8CF01F1180EB9ECAD
:101910000BF0E8CF02F1190EB9EC0BF0E8CF03F1B0
:10192000010103AFAEEF0CF058EC34F0160E0C6E64
:1019300000C10BF0A2EC0BF0170E0C6E01C10BF006
:10194000A2EC0BF0180E0C6E02C10BF0A2EC0BF027
:10195000190E0C6E03C10BF0A2EC0BF000C18AF162
:1019600001C18BF102C18CF103C18DF100C18EF177
:1019700001C18FF102C190F103C191F11A0EB9ECCE
:101980000BF0E8CF00F11B0EB9EC0BF0E8CF01F142
:101990001C0EB9EC0BF0E8CF02F11D0EB9EC0BF008
:1019A000E8CF03F1010103AF04EF0DF058EC34F080
:1019B0001A0E0C6E00C10BF0A2EC0BF01B0E0C6E9D
:1019C00001C10BF0A2EC0BF01C0E0C6E02C10BF06F
:1019D000A2EC0BF01D0E0C6E03C10BF0A2EC0BF091
:1019E0001A0EB9EC0BF0E8CF00F11B0EB9EC0BF0BE
:1019F000E8CF01F11C0EB9EC0BF0E8CF02F11D0E9F
:101A0000B9EC0BF0E8CF03F100C192F101C193F101
:101A100002C194F103C195F1240EAC6E900EAB6E31
:101A2000240EAC6E080EB86E000EB06E1F0EAF6EB8
:101A30000401806B816B0F01900EAB6E0F019D8ACC
:101A40000301806B816BC26B8B927EEC3AF07EEC73
:101A50003AF0880EB9EC0BF0E8CF00F1890EB9EC42
:101A60000BF0E8CF01F1010101AF4FEF0DF058ECA1
:101A700034F0880E0C6E00C10BF0A2EC0BF0890E56
:101A80000C6E01C10BF0A2EC0BF0880EB9EC0BF060
:101A9000E8CF00F1890EB9EC0BF0E8CF01F100C1FD
:101AA00040F601C141F602C142F603C143F6D6EC4D
:101AB0003DF05DEC38F0200EB9EC0BF0E8CF2FF5DF
:101AC00005012F51FF0AD8A46DEF0DF02F6B200EEA
:101AD0000C6E2FC50BF0A2EC0BF00501010E306F60
:101AE0003C0E316F250EB9EC0BF0E8CF00F1260E5D
:101AF000B9EC0BF0E8CF01F1270EB9EC0BF0E8CF11
:101B000002F1280EB9EC0BF0E8CF03F1010103AFAD
:101B1000A4EF0DF058EC34F0250E0C6E00C10BF064
:101B2000A2EC0BF0260E0C6E01C10BF0A2EC0BF038
:101B3000270E0C6E02C10BF0A2EC0BF0280E0C6EFF
:101B400003C10BF0A2EC0BF000C153F501C154F539
:101B500002C155F503C156F500C157F501C158F54D
:101B600002C159F503C15AF5290EB9EC0BF0E8CFC3
:101B70005BF505015C515B5DD8A05BC55CF50501BB
:101B80002F51020A0EE181B8D1EF0DF005015C2F53
:101B9000CEEF0DF05BC55CF5D1EF0DF081BA15EF1E
:101BA0003EF0210EB9EC0BF0E8CF00F1220EB9ECBB
:101BB0000BF0E8CF01F1230EB9EC0BF0E8CF02F106
:101BC000240EB9EC0BF0E8CF03F1010103AF17EFDE
:101BD0000EF058EC34F0210E0C6E00C10BF0A2ECAC
:101BE0000BF0220E0C6E01C10BF0A2EC0BF0230ED9
:101BF0000C6E02C10BF0A2EC0BF0240E0C6E03C1B4
:101C00000BF0A2EC0BF0210EB9EC0BF0E8CF00F1D9
:101C1000220EB9EC0BF0E8CF01F1230EB9EC0BF07A
:101C2000E8CF02F1240EB9EC0BF0E8CF03F100C1CC
:101C30005DF501C15EF502C15FF503C160F5A5EC7C
:101C400037F0A7EC36F0FFEC35F005012F51030A11
:101C500012E005012F51040A1DE005012F51050A6C
:101C600024E005012F51060A32E005012F51070A31
:101C700038E07AEF0EF0ACC500F101010F0E00174D
:101C800001010051000A36E001010051050A32E06D
:101C900077EF0EF0ACC500F101010F0E0017010146
:101CA0000051000A27E077EF0EF00501AC51000A61
:101CB00021E00501AC51150A1DE00501AC51300AC7
:101CC00019E00501AC51450A15E077EF0EF005016A
:101CD000AC51000A0FE00501AC51300A0BE077EF80
:101CE0000EF00501AC51000A05E077EF0EF081BA65
:101CF00015EF3EF090EC35F007900001F28EF28C7B
:101D000007B0BCEF2FF00FB069EF29F010BE69EFFC
:101D100029F012B869EF29F00FB80CEF23F0030196
:101D2000805181197F0BD8B4BCEF2FF013EE00F077
:101D300081517F0BE126812BE7CFE8FFE00BD8B480
:101D4000BCEF2FF023EE82F0C2513F0BD926E7CF34
:101D5000DFFFC22BDF50780AD8A4BCEF2FF007803A
:101D60008EC100F18FC101F190C102F191C103F167
:101D70000101040E046F000E056F000E066F000EC9
:101D8000076F5DEC33F000AFCFEF0EF00101030EF3
:101D90008E6F000E8F6F000E906F000E916F03011B
:101DA0008251720AD8B454EF29F08251520AD8B441
:101DB00054EF29F08251750AD8B454EF29F08251BA
:101DC000630AD8B476EF2CF08251690AD8B403EFD5
:101DD00026F082517A0AD8B416EF27F08251490AC8
:101DE000D8B4A2EF25F08251500AD8B4C0EF24F045
:101DF0008251700AD8B403EF25F08251540AD8B446
:101E00002EEF25F08251740AD8B474EF25F0825178
:101E1000410AD8B445EF0FF082516D0AD8B429EFCA
:101E200013F082514D0AD8B442EF13F08251730A75
:101E3000D8B484EF28F08251530AD8B4E9EF28F0DF
:101E400082514C0AD8B4A5EF1AF08251760AD8B460
:101E5000D1EF13F08251590AD8B47AEF12F0ADEFF6
:101E60002CF0040114EE00F080517F0BE12682C4B7
:101E7000E7FF802B120004010D0E826F31EC0FF092
:101E80000A0E826F31EC0FF012000401410E826FD6
:101E900031EC0FF003018351310AD8B49AEF11F0FD
:101EA00003018351320AD8B4F0EF10F003018351DB
:101EB000330AD8B479EF10F003018351340AD8B44F
:101EC00069EF0FF004013F0E826F31EC0FF0ABEFC2
:101ED0002CF0CC0EB9EC0BF0E8CF0BF004012C0E7B
:101EE000826F31EC0FF003018451310AD8B48DEFC9
:101EF0000FF003018451300AD8B48FEF0FF00301C3
:101F000084514D0AD8B499EF0FF003018451540A5B
:101F1000D8B4A0EF0FF0B7EF0FF08A8401D08A9405
:101F20000BAE04D00BAC02D00BBA21D0E00E0B12DA
:101F300018D01F0E0B168539E844E00B0B1211D098
:101F4000E00E0B1699EC34F085C332F186C333F101
:101F50000101296BA6EC34F01DEC34F000511F0B8D
:101F60000B12CC0E0C6E0BC00BF0A2EC0BF00401AC
:101F7000340E826F31EC0FF004012C0E826F31ECC5
:101F80000FF0CC0EB9EC0BF0E8CF19F08AB406D004
:101F90000401300E826F31EC0FF005D00401310ED8
:101FA000826F31EC0FF004012C0E826F31EC0FF0D8
:101FB0001938E840070BE8CF82F40401300E82277D
:101FC00031EC0FF004012C0E826F31EC0FF058EC65
:101FD00034F019501F0BE8CF00F1FBEC33F032C1A5
:101FE00082F40401300E822731EC0FF033C182F409
:101FF0000401300E822731EC0FF004012C0E826FA9
:1020000031EC0FF058EC34F02CC000F100AF0BD0E5
:10201000FF0E016FFF0E026FFF0E036F04012D0E06
:10202000826F31EC0FF0FBEC33F031C182F404012C
:10203000300E822731EC0FF032C182F40401300EF1
:10204000822731EC0FF033C182F40401300E822775
:1020500031EC0FF004012C0E826F31EC0FF058ECD4
:1020600034F02BC000F1FBEC33F031C182F40401F9
:10207000300E822731EC0FF032C182F40401300EB1
:10208000822731EC0FF033C182F40401300E822735
:1020900031EC0FF004012C0E826F31EC0FF058EC94
:1020A00034F02DC000F100AF0BD0FF0E016FFF0E1A
:1020B000026FFF0E036F04012D0E826F31EC0FF0E3
:1020C000FBEC33F031C182F40401300E822731EC95
:1020D0000FF032C182F40401300E822731EC0FF090
:1020E00033C182F40401300E822731EC0FF0ABEFE4
:1020F0002CF0CB0EB9EC0BF0E8CF0BF004012C0E5A
:10210000826F31EC0FF003018451450AD8B49DEF82
:1021100010F003018451440AD8B4A0EF10F0030179
:102120008451300AD8B4A3EF10F003018451310A6E
:10213000D8B4A7EF10F0B2EF10F00B9EACEF10F098
:102140000B8EACEF10F0FC0E0B16ACEF10F0FC0E8B
:102150000B160B80ACEF10F0CB0E0C6E0BC00BF01F
:10216000A2EC0BF00401330E826F31EC0FF004018E
:102170002C0E826F31EC0FF0CB0EB9EC0BF0E8CFE8
:1021800018F018BECBEF10F00401450E826F31EC51
:102190000FF0D0EF10F00401440E826F31EC0FF01D
:1021A00004012C0E826F31EC0FF00401300E826FAF
:1021B00031EC0FF004012C0E826F31EC0FF018B0EF
:1021C000E9EF10F00401300E826F31EC0FF0EEEF0A
:1021D00010F00401310E826F31EC0FF0ABEF2CF0F8
:1021E000CA0EB9EC0BF0E8CF0BF004012C0E826F95
:1021F00031EC0FF003018451450AD8B420EF11F0FF
:1022000003018451440AD8B423EF11F0030184512F
:102210004D0AD8B42CEF11F003018451410AD8B40F
:1022200026EF11F003018451460AD8B429EF11F0CA
:1022300003018451560AD8B434EF11F045EF11F080
:102240000B9E3FEF11F00B8E3FEF11F00B9C3FEF19
:1022500011F00B8C3FEF11F0F80E0B1685C3E8FF61
:10226000070B0B123FEF11F0C70E0B1685C3E8FFEB
:10227000070BE846E846E8460B123FEF11F0CA0E9E
:102280000C6E0BC00BF0A2EC0BF0CA0EB9EC0BF00D
:10229000E8CF17F00401320E826F31EC0FF0040129
:1022A0002C0E826F31EC0FF017BE5EEF11F00401BF
:1022B000450E826F31EC0FF063EF11F00401440E14
:1022C000826F31EC0FF004012C0E826F31EC0FF0B5
:1022D00017C0E8FF070BE8CF82F40401300E822715
:1022E00031EC0FF004012C0E826F31EC0FF017BCB3
:1022F00081EF11F00401410E826F31EC0FF086EF97
:1023000011F00401460E826F31EC0FF004012C0E27
:10231000826F31EC0FF017C0E8FF380BE842E8425B
:10232000E842E8CF82F40401300E822731EC0FF04E
:10233000ABEF2CF0C90EB9EC0BF0E8CF0BF00401B9
:102340002C0E826F31EC0FF003018451450AD8B492
:10235000B8EF11F003018451440AD8B4BBEF11F077
:10236000030184514D0AD8B4BEEF11F0CCEF11F047
:102370000B9EC6EF11F00B8EC6EF11F0F80E0B1688
:1023800085C3E8FF070B0B12C6EF11F0C90E0C6EE8
:102390000BC00BF0A2EC0BF00401310E826F31EC9C
:1023A0000FF004012C0E826F31EC0FF0C90EB9EC66
:1023B0000BF0E8CF16F016BE06D00401450E826F72
:1023C00031EC0FF005D00401440E826F31EC0FF0B8
:1023D00004012C0E826F31EC0FF016C0E8FF070BE2
:1023E000E8CF82F40401300E822731EC0FF00401B3
:1023F0002C0E826F31EC0FF0078058EC34F027C0C0
:10240000E8FF003B00430043030BFBEC33F033C118
:1024100082F40401300E822731EC0FF004012C0EFF
:10242000826F31EC0FF058EC34F027C001F1019FBE
:10243000019D28C000F10101FBEC33F02FC182F4B3
:102440000401300E822731EC0FF030C182F4040118
:10245000300E822731EC0FF031C182F40401300ECE
:10246000822731EC0FF032C182F40401300E822752
:1024700031EC0FF033C182F40401300E822731ECCD
:102480000FF004012C0E826F31EC0FF058EC34F099
:1024900029C001F12AC000F1D89001330033D8904F
:1024A000013300330101FBEC33F02FC182F404014E
:1024B000300E822731EC0FF030C182F40401300E6F
:1024C000822731EC0FF031C182F40401300E8227F3
:1024D00031EC0FF032C182F40401300E822731EC6E
:1024E0000FF033C182F40401300E822731EC0FF07B
:1024F000ABEF2CF0FC0EB9EC0BF0E8CF0BF00301C6
:102500008351520AD8B4B1EF12F003018351720A19
:10251000D8B4B4EF12F003018351500AD8B4B7EF26
:1025200012F003018351700AD8B4BAEF12F003011C
:102530008351550AD8B4BDEF12F003018351750AD7
:10254000D8B4C0EF12F003018351430AD8B4C9EFE5
:1025500012F003018351630AD8B4CCEF12F0D5EF27
:1025600012F00B90CFEF12F00B80CFEF12F00B9226
:10257000CFEF12F00B82CFEF12F00B94CFEF12F0EF
:102580000B84CFEF12F00B96CFEF12F00B86CFEF4C
:1025900012F00B98CFEF12F00B88CFEF12F0FC0E79
:1025A0000C6E0BC00BF0A2EC0BF00401590E826F05
:1025B00031EC0FF01190119211941198FC0EB9ECBE
:1025C0000BF0E8CF0BF00BA011800BA211820BA433
:1025D00011840BA8118811A0F5EF12F00401520E1E
:1025E000826F31EC0FF0FAEF12F00401720E826F7D
:1025F00031EC0FF011A804EF13F00401430E826FC9
:1026000031EC0FF009EF13F00401630E826F31EC2F
:102610000FF011A213EF13F00401500E826F31EC92
:102620000FF018EF13F00401700E826F31EC0FF011
:1026300011A422EF13F00401550E826F31EC0FF05C
:1026400027EF13F00401750E826F31EC0FF0ABEF42
:102650002CF004016D0E826F31EC0FF003018351F9
:10266000300AD8B481EF13F003018351310AD8B492
:1026700094EF13F003018351320AD8B4A7EF13F09B
:10268000ADEF2CF004014D0E826F31EC0FF099ECA0
:1026900034F084C331F185C332F186C333F10101D3
:1026A000296BA6EC34F01DEC34F003018351300AA1
:1026B000D8B469EF13F003018351310AD8B471EF34
:1026C00013F003018351320AD8B479EF13F0ADEF60
:1026D0002CF0FD0E0C6E00C10BF0A2EC0BF081EFA4
:1026E00013F0FE0E0C6E00C10BF0A2EC0BF094EF99
:1026F00013F0FF0E0C6E00C10BF0A2EC0BF0A7EF75
:1027000013F00401300E826F31EC0FF004012C0E37
:10271000826F31EC0FF058EC34F0FD0EB9EC0BF099
:10272000E8CF00F1B8EF13F00401310E826F31EC05
:102730000FF004012C0E826F31EC0FF058EC34F0E6
:10274000FE0EB9EC0BF0E8CF00F1B8EF13F0040186
:10275000320E826F31EC0FF058EC34F004012C0E85
:10276000826F31EC0FF0FF0EB9EC0BF0E8CF00F107
:10277000FBEC33F031C182F40401300E822731ECDE
:102780000FF032C182F40401300E822731EC0FF0D9
:1027900033C182F40401300E822731EC0FF0ABEF2D
:1027A0002CF003018351300AD8B476EF15F0030101
:1027B0008351310AD8B4ADEF15F003018351320AC9
:1027C000D8B462EF17F003018351330AD8B417EF7E
:1027D00019F003018351340AD8B4BDEF19F0030195
:1027E0008351730AD8B458EF14F003018351760A69
:1027F000D8B45AEF14F003018351740AD8B445EFEA
:1028000014F003018351540AD8B40AEF14F0D8A489
:10281000ADEF2CF00401760E826F31EC0FF0040165
:10282000540E826F31EC0FF007840001880E0C6E9D
:1028300099EC34F02981030184512D0AD8B423EF97
:1028400014F00101299185C32FF186C330F187C3AC
:1028500031F188C332F189C333F1A6EC34F01DECB9
:1028600034F000C10BF0A2EC0BF001C10BF0A2ECB4
:102870000BF0880EB9EC0BF0E8CF40F6890EB9ECFE
:102880000BF0E8CF41F650EF14F00401760E826FA2
:1028900031EC0FF00401740E826F31EC0FF00784FD
:1028A0000001880E0C6EC0EC0BF007946DEF23F066
:1028B00058EC14F00401760E826F31EC0FF0040135
:1028C000760E826F31EC0FF00784D5EC30F0040106
:1028D0002C0E826F31EC0FF00101036B026B3BC6D3
:1028E00001F13AC600F101AF7BEF14F00101FF0ED8
:1028F000026FFF0E036FFBEC33F0296782EF14F0D9
:1029000087EF14F004012D0E826F31EC0FF02FC110
:1029100082F40401300E822731EC0FF030C182F4D2
:102920000401300E822731EC0FF031C182F4040132
:10293000300E822731EC0FF032C182F40401300EE8
:10294000822731EC0FF033C182F40401300E82276C
:1029500031EC0FF004012C0E826F31EC0FF001010D
:10296000036B026B3DC601F13CC600F101AFBEEF47
:1029700014F00101FF0E026FFF0E036FFBEC33F04A
:102980002967C5EF14F0CAEF14F004012D0E826F11
:1029900031EC0FF02FC182F40401300E822731ECAC
:1029A0000FF030C182F40401300E822731EC0FF0B9
:1029B00031C182F40401300E822731EC0FF032C1B4
:1029C00082F40401300E822731EC0FF033C182F41F
:1029D0000401300E822731EC0FF004012C0E826FBF
:1029E00031EC0FF00101036B026B3FC601F13EC6F3
:1029F00000F101AF01EF15F00101FF0E026FFF0EB4
:102A0000036FFBEC33F0296708EF15F00DEF15F0BD
:102A100004012D0E826F31EC0FF02FC182F40401FE
:102A2000300E822731EC0FF030C182F40401300EF9
:102A3000822731EC0FF031C182F40401300E82277D
:102A400031EC0FF032C182F40401300E822731ECF8
:102A50000FF033C182F40401300E822731EC0FF005
:102A600004012C0E826F31EC0FF00101036B026B3D
:102A700037C601F136C600F101AF44EF15F0010190
:102A8000FF0E026FFF0E036FFBEC33F029674BEF75
:102A900015F050EF15F004012D0E826F31EC0FF0A0
:102AA0002FC182F40401300E822731EC0FF030C1C7
:102AB00082F40401300E822731EC0FF031C182F430
:102AC0000401300E822731EC0FF032C182F4040190
:102AD000300E822731EC0FF033C182F40401300E46
:102AE000822731EC0FF007946DEF23F00401760E8E
:102AF000826F31EC0FF00401300E826F31EC0FF079
:102B000004012C0E826F31EC0FF0C6EC34F058EC5F
:102B100034F000C600F101C601F1FBEC33F030C126
:102B200082F40401300E822731EC0FF031C182F4BF
:102B30000401300E822731EC0FF032C182F404011F
:102B4000300E822731EC0FF033C182F40401300ED5
:102B5000822731EC0FF06DEF23F00401760E826FC7
:102B600031EC0FF00401310E826F31EC0FF007846D
:102B70000101036B026B02C600F103C601F101AF54
:102B8000C6EF15F0FF0E026FFF0E036F0101076B1A
:102B9000066B04C604F105C605F105AFD4EF15F0C8
:102BA000FF0E066FFF0E076F62EC33F00101076B3B
:102BB000066B06C604F107C605F105AFE4EF15F094
:102BC000FF0E066FFF0E076F62EC33F00101076B1B
:102BD000066B08C604F109C605F105AFF4EF15F060
:102BE000FF0E066FFF0E076F62EC33F0D890010105
:102BF0000333023301330033D8900101033302332E
:102C00000133003304012C0E826F31EC0FF001010F
:102C1000036B026B01C101F100C100F101AF16EFBE
:102C200016F00101FF0E026FFF0E036FFBEC33F095
:102C300029671DEF16F022EF16F004012D0E826FAA
:102C400031EC0FF02FC182F40401300E822731ECF9
:102C50000FF030C182F40401300E822731EC0FF006
:102C600031C182F40401300E822731EC0FF032C101
:102C700082F40401300E822731EC0FF033C182F46C
:102C80000401300E822731EC0FF00101036B026B5F
:102C90000AC600F10BC601F101AF53EF16F0FF0EAB
:102CA000026FFF0E036F0101076B066B0CC604F188
:102CB0000DC605F105AF61EF16F0FF0E066FFF0EB2
:102CC000076F62EC33F00101076B066B0EC604F16F
:102CD0000FC605F105AF71EF16F0FF0E066FFF0E80
:102CE000076F62EC33F00101076B066B10C604F14D
:102CF00011C605F105AF81EF16F0FF0E066FFF0E4E
:102D0000076F62EC33F0D8900101033302330133D3
:102D10000033D8900101033302330133003304013F
:102D20002C0E826F31EC0FF00101036B026B01C1BD
:102D300001F100C100F101AFA3EF16F00101FF0E98
:102D4000026FFF0E036FFBEC33F02967AAEF16F05A
:102D5000AFEF16F004012D0E826F31EC0FF02FC192
:102D600082F40401300E822731EC0FF030C182F47E
:102D70000401300E822731EC0FF031C182F40401DE
:102D8000300E822731EC0FF032C182F40401300E94
:102D9000822731EC0FF033C182F40401300E822718
:102DA00031EC0FF00101036B026B12C600F113C688
:102DB00001F101AFE0EF16F0FF0E026FFF0E036F9F
:102DC0000101076B066B14C604F115C605F105AFCA
:102DD000EEEF16F0FF0E066FFF0E076F62EC33F09A
:102DE0000101076B066B16C604F117C605F105AFA6
:102DF000FEEF16F0FF0E066FFF0E076F62EC33F06A
:102E00000101076B066B18C604F119C605F105AF81
:102E10000EEF17F0FF0E066FFF0E076F62EC33F038
:102E2000D89001010333023301330033D8900101FC
:102E3000033302330133003304012C0E826F31EC73
:102E40000FF00101036B026B01C101F100C100F140
:102E500001AF30EF17F00101FF0E026FFF0E036F9D
:102E6000FBEC33F0296737EF17F03CEF17F0040164
:102E70002D0E826F31EC0FF02FC182F40401300E61
:102E8000822731EC0FF030C182F40401300E82272A
:102E900031EC0FF031C182F40401300E822731ECA5
:102EA0000FF032C182F40401300E822731EC0FF0B2
:102EB00033C182F40401300E822731EC0FF0079405
:102EC0006DEF23F00401760E826F31EC0FF00401F8
:102ED000320E826F31EC0FF007840101036B026B3D
:102EE0001AC600F11BC601F101AF7BEF17F0FF0E10
:102EF000026FFF0E036F0101076B066B1CC604F126
:102F00001DC605F105AF89EF17F0FF0E066FFF0E26
:102F1000076F62EC33F00101076B066B1EC604F10C
:102F20001FC605F105AF99EF17F0FF0E066FFF0EF4
:102F3000076F62EC33F00101076B066B20C604F1EA
:102F400021C605F105AFA9EF17F0FF0E066FFF0EC2
:102F5000076F62EC33F0D890010103330233013381
:102F60000033D890010103330233013300330401ED
:102F70002C0E826F31EC0FF00101036B026B01C16B
:102F800001F100C100F101AFCBEF17F00101FF0E1D
:102F9000026FFF0E036FFBEC33F02967D2EF17F0DF
:102FA000D7EF17F004012D0E826F31EC0FF02FC117
:102FB00082F40401300E822731EC0FF030C182F42C
:102FC0000401300E822731EC0FF031C182F404018C
:102FD000300E822731EC0FF032C182F40401300E42
:102FE000822731EC0FF033C182F40401300E8227C6
:102FF00031EC0FF00101036B026B22C600F123C616
:1030000001F101AF08EF18F0FF0E026FFF0E036F22
:103010000101076B066B24C604F125C605F105AF57
:1030200016EF18F0FF0E066FFF0E076F62EC33F01D
:103030000101076B066B26C604F127C605F105AF33
:1030400026EF18F0FF0E066FFF0E076F62EC33F0ED
:103050000101076B066B28C604F129C605F105AF0F
:1030600036EF18F0FF0E066FFF0E076F62EC33F0BD
:10307000D89001010333023301330033D8900101AA
:10308000033302330133003304012C0E826F31EC21
:103090000FF00101036B026B01C101F100C100F1EE
:1030A00001AF58EF18F00101FF0E026FFF0E036F22
:1030B000FBEC33F029675FEF18F064EF18F00401C0
:1030C0002D0E826F31EC0FF02FC182F40401300E0F
:1030D000822731EC0FF030C182F40401300E8227D8
:1030E00031EC0FF031C182F40401300E822731EC53
:1030F0000FF032C182F40401300E822731EC0FF060
:1031000033C182F40401300E822731EC0FF001014B
:10311000036B026B2AC600F12BC601F101AF95EFDC
:1031200018F0FF0E026FFF0E036F0101076B066BB5
:103130002CC604F12DC605F105AFA3EF18F0FF0E64
:10314000066FFF0E076F62EC33F00101076B066B31
:103150002EC604F12FC605F105AFB3EF18F0FF0E30
:10316000066FFF0E076F62EC33F00101076B066B11
:1031700030C604F131C605F105AFC3EF18F0FF0EFC
:10318000066FFF0E076F62EC33F0D8900101033336
:10319000023301330033D89001010333023301338A
:1031A000003304012C0E826F31EC0FF00101036B30
:1031B000026B01C101F100C100F101AFE5EF18F0B0
:1031C0000101FF0E026FFF0E036FFBEC33F0296766
:1031D000ECEF18F0F1EF18F004012D0E826F31ECD6
:1031E0000FF02FC182F40401300E822731EC0FF072
:1031F00030C182F40401300E822731EC0FF031C16E
:1032000082F40401300E822731EC0FF032C182F4D7
:103210000401300E822731EC0FF033C182F4040137
:10322000300E822731EC0FF007946DEF23F004018C
:10323000760E826F31EC0FF00401330E826F31ECA9
:103240000FF004012C0E826F31EC0FF085C382F475
:1032500031EC0FF0640E0D6E03018551320A02E16C
:103260006A0E0D6E03018551330A02E1700E0D6E78
:1032700003018551340A02E1760E0D6E030185517A
:10328000350A02E17C0E0D6E03018551360A02E11A
:10329000820E0D6E03018651780A65E00DC00CF0B8
:1032A00099EC34F02981030187512D0AD8B45BEFE2
:1032B00019F00101299188C32FF189C330F18AC324
:1032C00031F18BC332F18CC333F1A6EC34F01DEC39
:1032D00034F000C10BF0A2EC0BF001C10BF0A2EC3A
:1032E0000BF099EC34F0298103018E512D0AD8B4EA
:1032F0007CEF19F0010129918FC32FF190C330F1B8
:1033000091C331F192C332F193C333F1A6EC34F09F
:103310001DEC34F000C10BF0A2EC0BF001C10BF07E
:10332000A2EC0BF099EC34F02981030195512D0AA0
:10333000D8B49DEF19F00101299196C32FF197C3DD
:1033400030F198C331F199C332F19AC333F1A6EC4D
:1033500034F01DEC34F000C10BF0A2EC0BF001C115
:103360000BF0A2EC0BF00DC00CF0C0EC0BF0C0ECBD
:103370000BF0C0EC0BF06DEF23F00401760E826FC2
:1033800031EC0FF00401340E826F31EC0FF00301C9
:103390008451780AD8B495EF1AF03E0E0C6E99EC71
:1033A00034F02981030185512D0AD8B4DAEF19F0E0
:1033B0000101299186C32FF187C330F188C331F110
:1033C00089C332F18AC333F1A6EC34F01DEC34F03A
:1033D00000C10BF0A2EC0BF001C10BF0A2EC0BF062
:1033E00099EC34F0298103018C512D0AD8B4FBEFFC
:1033F00019F0010129918DC32FF18EC330F18FC3D4
:1034000031F190C332F191C333F1A6EC34F01DECED
:1034100034F000C10BF0A2EC0BF001C10BF0A2ECF8
:103420000BF099EC34F02981030193512D0AD8B4A3
:103430001CEF1AF00101299194C32FF195C330F1CB
:1034400096C331F197C332F198C333F1A6EC34F04F
:103450001DEC34F000C10BF0A2EC0BF001C10BF03D
:10346000A2EC0BF099EC34F0298103019A512D0A5A
:10347000D8B43DEF1AF0010129919BC32FF19CC3F1
:1034800030F19DC331F19EC332F19FC333F1A6ECFD
:1034900034F01DEC34F000C10BF0A2EC0BF001C1D4
:1034A0000BF0A2EC0BF099EC34F029810301A1514F
:1034B0002D0AD8B45EEF1AF001012991A2C32FF1B1
:1034C000A3C330F1A4C331F1A5C332F1A6C333F1D4
:1034D000A6EC34F01DEC34F000C10BF0A2EC0BF0C4
:1034E00001C10BF0A2EC0BF099EC34F0298103013F
:1034F000A8512D0AD8B47FEF1AF001012991A9C370
:103500002FF1AAC330F1ABC331F1ACC332F1ADC37B
:1035100033F1A6EC34F01DEC34F000C10BF0A2EC5A
:103520000BF001C10BF0A2EC0BF03E0E0C6EC0ECE8
:103530000BF0C0EC0BF0C0EC0BF0C0EC0BF0C0ECEF
:103540000BF0C0EC0BF06DEF23F003018351300A58
:10355000D8B410EF1EF003018351310AD8B43DEF07
:103560001FF003018351320AD8B4ABEF1FF00301FF
:103570008351330AD8B4BBEF1FF003018351340ADF
:10358000D8B4CBEF1FF003018351350AD8B411EF43
:1035900023F003018351360AD8B43FEF23F003012F
:1035A0008351370AD8B472EF1DF003018351460AE4
:1035B000D8B465EF22F0030183514D0AD8B4EBEF84
:1035C0001BF0030183516D0AD8B405EF1CF0030111
:1035D00083515A0AD8B4B7EF1EF003018351490A48
:1035E000D8B43FEF24F003018351500AD8B471EFEF
:1035F00023F003018351540AD8B4EAEF23F0030106
:103600008351630AD8B425EF1CF003018351430AA8
:10361000D8B41DEF1DF003018351730AD8B423EF12
:103620001CF003018351610AD8B438EF1BF0030189
:103630008351650AD8B460EF1EF003018351450A37
:10364000D8B46EEF1EF003018351620AD8B47CEF48
:103650001EF003018351420AD8B48AEF1EF0030121
:103660008351760AD8B498EF1EF0D8A4ADEF2CF0B1
:1036700004014C0E826F31EC0FF00401610E826F79
:1036800031EC0FF0A7EC36F004012C0E826F31EC18
:103690000FF058EC34F0ABC500F10101FBEC33F056
:1036A00031C182F40401300E822731EC0FF032C1B7
:1036B00082F40401300E822731EC0FF033C182F422
:1036C0000401300E822731EC0FF004012C0E826FC2
:1036D00031EC0FF058EC34F0ACC500F10101FBEC1B
:1036E00033F031C182F40401300E822731EC0FF047
:1036F00032C182F40401300E822731EC0FF033C165
:1037000082F40401300E822731EC0FF004012C0EFC
:10371000826F31EC0FF058EC34F0ADC500F10101CF
:10372000FBEC33F031C182F40401300E822731EC1E
:103730000FF032C182F40401300E822731EC0FF019
:1037400033C182F40401300E822731EC0FF0040102
:103750002C0E826F31EC0FF058EC34F0AEC500F156
:103760000101FBEC33F031C182F40401300E8227F9
:1037700031EC0FF032C182F40401300E822731ECBB
:103780000FF033C182F40401300E822731EC0FF0C8
:1037900004012C0E826F31EC0FF058EC34F0B2C5FE
:1037A00000F10101FBEC33F031C182F40401300E71
:1037B000822731EC0FF032C182F40401300E8227EF
:1037C00031EC0FF033C182F40401300E822731EC6A
:1037D0000FF06DEF23F099EC34F084C333F1A6ECD5
:1037E00034F01DEC34F0200E0C6E00C10BF0A2EC96
:1037F0000BF000C12FF505012F51000A06E005016D
:103800002F51010A02E041EC37F004014C0E826FA7
:1038100031EC0FF004014D0E826F31EC0FF004011A
:103820002C0E826F31EC0FF058EC34F02FC500F104
:10383000FBEC33F033C182F40401300E822731EC0B
:103840000FF06DEF23F015EF3EF004014C0E826F88
:1038500031EC0FF00401630E826F31EC0FF0FFECDE
:1038600035F004012C0E826F31EC0FF03AEC1CF0B5
:103870006DEF23F058EC34F0B1C500F10101003BCD
:103880000F0E0017FBEC33F033C182F40401300E4D
:10389000822731EC0FF0B1C500F101010F0E0101DB
:1038A0000017FBEC33F033C182F40401300E8227A1
:1038B00031EC0FF004012D0E826F31EC0FF0B0C52A
:1038C00000F10101003B0F0E0017FBEC33F033C198
:1038D00082F40401300E822731EC0FF0B0C500F104
:1038E00001010F0E01010017FBEC33F033C182F42C
:1038F0000401300E822731EC0FF004012D0E826F8F
:1039000031EC0FF0AFC500F10101003B0F0E0017C5
:10391000FBEC33F033C182F40401300E822731EC2A
:103920000FF0AFC500F101010F0E01010017FBEC14
:1039300033F033C182F40401300E822731EC0FF0F2
:103940000401200E826F31EC0FF0AEC500F10F0EB6
:1039500001010017FBEC33F033C182F40401300E97
:10396000822731EC0FF00401200E826F31EC0FF052
:10397000ADC500F101010101003B0F0E0017FBEC8A
:1039800033F033C182F40401300E822731EC0FF0A2
:10399000ADC500F101010F0E01010017FBEC33F082
:1039A00033C182F40401300E822731EC0FF00401A0
:1039B0003A0E826F31EC0FF0ACC500F10101003B13
:1039C0000F0E0017FBEC33F033C182F40401300E0C
:1039D000822731EC0FF0ACC500F101010F0E01019F
:1039E0000017FBEC33F033C182F40401300E822760
:1039F00031EC0FF004013A0E826F31EC0FF0ABC5E1
:103A000000F10101003B0F0E0017FBEC33F033C156
:103A100082F40401300E822731EC0FF0ABC500F1C7
:103A200001010F0E0017FBEC33F033C182F40401E7
:103A3000300E822731EC0FF0120084C3E8FF0F0B29
:103A4000E83AE8CFB1F585C3E8FF0F0B0501B113E4
:103A500087C3E8FF0F0BE83AE8CFB0F588C3E8FF6B
:103A60000F0B0501B0138AC3E8FF0F0BE83AE8CF4C
:103A7000AFF58BC3E8FF0F0B0501AF138DC3E8FF54
:103A80000F0BE8CFAEF58FC3E8FF0F0BE83AE8CF96
:103A9000ADF590C3E8FF0F0B0501AD1392C3E8FF2E
:103AA0000F0BE83AE8CFACF593C3E8FF0F0B050125
:103AB000AC1395C3E8FF0F0BE83AE8CFABF596C31C
:103AC000E8FF0F0B0501AB135AEC36F004014C0E66
:103AD000826F31EC0FF00401430E826F31EC0FF076
:103AE0002FEF1CF0078404014C0E826F31EC0FF0B5
:103AF0000401370E826F31EC0FF004012C0E826F3F
:103B000031EC0FF005012E51130A06E005012E518C
:103B1000170A0DE00DEF1EF00101000E006F000E00
:103B2000016F100E026F000E036FA0EF1DF0010178
:103B3000000E006F000E016F000E026F010E036F8A
:103B4000FBEC33F02AC182F40401300E822731EC01
:103B50000FF02BC182F40401300E822731EC0FF0FC
:103B60002CC182F40401300E822731EC0FF02DC1FC
:103B700082F40401300E822731EC0FF02EC182F462
:103B80000401300E822731EC0FF02FC182F40401C2
:103B9000300E822731EC0FF030C182F40401300E78
:103BA000822731EC0FF031C182F40401300E8227FC
:103BB00031EC0FF032C182F40401300E822731EC77
:103BC0000FF033C182F40401300E822731EC0FF084
:103BD00004012C0E826F31EC0FF00101200E006FFA
:103BE000000E016F000E026F000E036FFBEC33F04E
:103BF00031C182F40401300E822731EC0FF032C162
:103C000082F40401300E822731EC0FF033C182F4CC
:103C10000401300E822731EC0FF007946DEF23F092
:103C20000784D6EC3DF058EC34F02DC500F1FBECE8
:103C300033F004014C0E826F31EC0FF00401300EB2
:103C4000826F31EC0FF004012C0E826F31EC0FF01B
:103C500031C182F40401300E822731EC0FF032C101
:103C600082F40401300E822731EC0FF033C182F46C
:103C70000401300E822731EC0FF004012C0E826F0C
:103C800031EC0FF058EC34F02EC500F1FBEC33F0C2
:103C900031C182F40401300E822731EC0FF032C1C1
:103CA00082F40401300E822731EC0FF033C182F42C
:103CB0000401300E822731EC0FF007946DEF23F0F2
:103CC00004014C0E826F31EC0FF00401650E826F1F
:103CD00031EC0FF001EC38F06DEF23F004014C0EE5
:103CE000826F31EC0FF00401450E826F31EC0FF062
:103CF00018EC38F06DEF23F004014C0E826F31ECBC
:103D00000FF00401620E826F31EC0FF046EC38F0D8
:103D10006DEF23F004014C0E826F31EC0FF00401C3
:103D2000420E826F31EC0FF02FEC38F06DEF23F084
:103D300004014C0E826F31EC0FF00401760E826F9D
:103D400031EC0FF004012C0E826F31EC0FF010A853
:103D500007D00401310E826F31EC0FF06DEF23F0CC
:103D60000401300E826F31EC0FF06DEF23F004018F
:103D70004C0E826F31EC0FF004015A0E826F31EC61
:103D80000FF004012C0E826F31EC0FF0D6EC3DF0F9
:103D900058EC34F005012E51130A06E005012E51AE
:103DA000170A0DE0E8EF1EF00101000E006F000E93
:103DB000016F100E026F000E036FE8EF1EF001019D
:103DC000000E006F000E016F000E026F010E036FF8
:103DD0000101200E046F000E056F000E066F000E2D
:103DE000076F8EEC33F0FBEC33F02AC182F4040150
:103DF000300E822731EC0FF02BC182F40401300E1B
:103E0000822731EC0FF02CC182F40401300E82279E
:103E100031EC0FF02DC182F40401300E822731EC19
:103E20000FF02EC182F40401300E822731EC0FF026
:103E30002FC182F40401300E822731EC0FF030C123
:103E400082F40401300E822731EC0FF031C182F48C
:103E50000401300E822731EC0FF032C182F40401EC
:103E6000300E822731EC0FF033C182F40401300EA2
:103E7000822731EC0FF06DEF23F0078404014C0E24
:103E8000826F31EC0FF00401310E826F31EC0FF0D4
:103E900004012C0E826F31EC0FF025C500F126C510
:103EA00001F127C502F128C503F10101200E046FBD
:103EB000000E056F000E066F000E076F8EEC33F0DC
:103EC000FBEC33F02AC182F40401300E822731EC7E
:103ED0000FF02BC182F40401300E822731EC0FF079
:103EE0002CC182F40401300E822731EC0FF02DC179
:103EF00082F40401300E822731EC0FF02EC182F4DF
:103F00000401300E822731EC0FF02FC182F404013E
:103F1000300E822731EC0FF030C182F40401300EF4
:103F2000822731EC0FF031C182F40401300E822778
:103F300031EC0FF032C182F40401300E822731ECF3
:103F40000FF033C182F40401300E822731EC0FF000
:103F500007946DEF23F0078404014C0E826F31EC5F
:103F60000FF00401320E826F31EC0FF034EC3AF0B6
:103F700007946DEF23F0078404014C0E826F31EC3F
:103F80000FF00401330E826F31EC0FF091EC3AF038
:103F9000079448EF1FF0078404014C0E826F31EC48
:103FA0000FF00401340E826F31EC0FF004012C0E7F
:103FB000826F31EC0FF099EC34F084C32AF185C3A1
:103FC0002BF186C32CF187C32DF188C32EF189C351
:103FD0002FF18AC330F18BC331F18CC332F18DC321
:103FE00033F10101296BA6EC34F01DEC34F0200E06
:103FF000046F000E056F000E066F000E076F6EEC6B
:1040000033F000C121F501C122F502C123F503C13E
:1040100024F589EC3DF034C5ABF535C5ACF536C5B6
:10402000ADF537C5AEF538C5AFF539C5B0F53AC50C
:10403000B1F53AEC1CF004012C0E826F31EC0FF05C
:104040003BC500F13CC501F13DC502F13EC503F1A0
:104050000101000E046F000E056F010E066F000EC9
:10406000076F8EEC33F0FBEC33F029673AEF20F06A
:104070003FEF20F004012D0E826F31EC0FF030C1C4
:1040800082F40401300E822731EC0FF031C182F44A
:104090000401300E822731EC0FF004012E0E826FE6
:1040A00031EC0FF032C182F40401300E822731EC82
:1040B0000FF033C182F40401300E822731EC0FF08F
:1040C00004012C0E826F31EC0FF058EC34F03FC538
:1040D00000F140C501F1D7EC2DF004012C0E826FE8
:1040E00031EC0FF058EC34F041C500F1FBEC33F04B
:1040F00031C182F40401300E822731EC0FF032C15D
:1041000082F40401300E822731EC0FF033C182F4C7
:104110000401300E822731EC0FF004012C0E826F67
:1041200031EC0FF00101036B026B48C501F147C58B
:1041300000F101AFA1EF20F00101FF0E026FFF0EB1
:10414000036FFBEC33F02967A8EF20F0ADEF20F010
:1041500004012D0E826F31EC0FF02FC182F40401A7
:10416000300E822731EC0FF030C182F40401300EA2
:10417000822731EC0FF031C182F40401300E822726
:1041800031EC0FF032C182F40401300E822731ECA1
:104190000FF033C182F40401300E822731EC0FF0AE
:1041A00004012C0E826F31EC0FF00101036B026BE6
:1041B0004AC501F149C500F101AFE4EF20F001016A
:1041C000FF0E026FFF0E036FFBEC33F02967EBEF7E
:1041D00020F0F0EF20F004012D0E826F31EC0FF093
:1041E0002FC182F40401300E822731EC0FF030C170
:1041F00082F40401300E822731EC0FF031C182F4D9
:104200000401300E822731EC0FF032C182F4040138
:10421000300E822731EC0FF033C182F40401300EEE
:10422000822731EC0FF004012C0E826F31EC0FF07D
:104230000101036B026B4CC501F14BC500F101AFED
:1042400027EF21F00101FF0E026FFF0E036FFBEC61
:1042500033F029672EEF21F033EF21F004012D0E0A
:10426000826F31EC0FF02FC182F40401300E8227EF
:1042700031EC0FF030C182F40401300E822731ECB2
:104280000FF031C182F40401300E822731EC0FF0BF
:1042900032C182F40401300E822731EC0FF033C1B9
:1042A00082F40401300E822731EC0FF004012C0E51
:1042B000826F31EC0FF00101036B026B4EC501F10F
:1042C0004DC500F101AF6AEF21F00101FF0E026F51
:1042D000FF0E036FFBEC33F0296771EF21F076EFEF
:1042E00021F004012D0E826F31EC0FF02FC182F40A
:1042F0000401300E822731EC0FF030C182F404014A
:10430000300E822731EC0FF031C182F40401300EFF
:10431000822731EC0FF032C182F40401300E822783
:1043200031EC0FF033C182F40401300E822731ECFE
:104330000FF004012C0E826F31EC0FF00101036BC2
:10434000026B50C501F14FC500F101AFADEF21F097
:104350000101FF0E026FFF0E036FFBEC33F02967C4
:10436000B4EF21F0B9EF21F004012D0E826F31EC92
:104370000FF02FC182F40401300E822731EC0FF0D0
:1043800030C182F40401300E822731EC0FF031C1CC
:1043900082F40401300E822731EC0FF032C182F436
:1043A0000401300E822731EC0FF033C182F4040196
:1043B000300E822731EC0FF004012C0E826F31ECAD
:1043C0000FF00101036B026B52C501F151C500F101
:1043D00001AFF0EF21F00101FF0E026FFF0E036F3E
:1043E000FBEC33F02967F7EF21F0FCEF21F004013B
:1043F0002D0E826F31EC0FF02FC182F40401300ECC
:10440000822731EC0FF030C182F40401300E822794
:1044100031EC0FF031C182F40401300E822731EC0F
:104420000FF032C182F40401300E822731EC0FF01C
:1044300033C182F40401300E822731EC0FF0040105
:104440002C0E826F31EC0FF00101036B026B46C53D
:1044500001F145C500F101AF33EF22F00101FF0E7C
:10446000026FFF0E036FFBEC33F029673AEF22F087
:104470003FEF22F004012D0E826F31EC0FF02FC1BF
:1044800082F40401300E822731EC0FF030C182F447
:104490000401300E822731EC0FF031C182F40401A7
:1044A000300E822731EC0FF032C182F40401300E5D
:1044B000822731EC0FF033C182F40401300E8227E1
:1044C00031EC0FF007946DEF23F099EC34F085C3D5
:1044D0002AF186C32BF187C32CF188C32DF189C340
:1044E0002EF18AC32FF18BC330F18CC331F18DC310
:1044F00032F18EC333F10101296BA6EC34F01DECCF
:1045000034F00101010E046F000E056F000E066FFE
:10451000000E076F5DEC33F0100E046F000E056F98
:10452000000E066F000E076F6EEC33F000C129F528
:1045300001C12AF502C12BF503C12CF5BBEC39F002
:1045400004014C0E826F31EC0FF00401460E826FB5
:1045500031EC0FF004012C0E826F31EC0FF025C509
:1045600000F126C501F127C502F128C503F10101BB
:10457000100E046F000E056F000E066F000E076F21
:104580008EEC33F0FBEC33F02AC182F40401300EE0
:10459000822731EC0FF02BC182F40401300E822708
:1045A00031EC0FF02CC182F40401300E822731EC83
:1045B0000FF02DC182F40401300E822731EC0FF090
:1045C0002EC182F40401300E822731EC0FF02FC18E
:1045D00082F40401300E822731EC0FF030C182F4F6
:1045E0000401300E822731EC0FF031C182F4040156
:1045F000300E822731EC0FF032C182F40401300E0C
:10460000822731EC0FF033C182F40401300E82278F
:1046100031EC0FF06DEF23F00F9891EC3AF0ADEF25
:104620002CF004014C0E826F31EC0FF00401350EBA
:10463000826F31EC0FF004012C0E826F31EC0FF021
:1046400058EC34F00784B5C500F10794FBEC33F067
:1046500031C182F40401300E822731EC0FF032C1F7
:1046600082F40401300E822731EC0FF033C182F462
:104670000401300E822731EC0FF06DEF23F054EC83
:104680003AF058EC34F033C500F1FBEC33F00401A0
:104690004C0E826F31EC0FF00401360E826F31EC5C
:1046A0000FF004012C0E826F31EC0FF031C182F457
:1046B0000401300E822731EC0FF032C182F4040184
:1046C000300E822731EC0FF033C182F40401300E3A
:1046D000822731EC0FF06DEF23F03BEC0FF0ADEFE4
:1046E0002CF004014C0E826F31EC0FF00401500EDF
:1046F000826F31EC0FF004012C0E826F31EC0FF061
:1047000085C32AF186C32BF187C32CF188C32DF111
:1047100089C32EF18AC32FF18BC330F18CC331F1E1
:104720008DC332F18EC333F10101A6EC34F01DECE0
:1047300034F003018451530A0DE0030184514D0A02
:1047400038E00401780E826F31EC0FF03BEC0FF093
:10475000ADEF2CF00401530E826F31EC0FF0250EFB
:104760000C6E00C10BF0A2EC0BF0260E0C6E01C11A
:104770000BF0A2EC0BF0270E0C6E02C10BF0A2ECBA
:104780000BF0280E0C6E03C10BF0A2EC0BF000C175
:1047900053F501C154F502C155F503C156F500C1E9
:1047A00057F501C158F502C159F503C15AF54EEF4D
:1047B00024F004014D0E826F31EC0FF0290E0C6EC7
:1047C00000C10BF0A2EC0BF000C15BF500C15CF581
:1047D0004EEF24F004014C0E826F31EC0FF0040117
:1047E000540E826F31EC0FF004012C0E826F31EC0D
:1047F0000FF084C32AF185C32BF186C32CF187C344
:104800002DF188C32EF189C32FF18AC330F18BC3F8
:1048100031F18DC332F18EC333F10101A6EC34F0D6
:104820001DEC34F00101000E046F000E056F010E47
:10483000066F000E076F6EEC33F0210E0C6E00C198
:104840000BF0A2EC0BF0220E0C6E01C10BF0A2ECEF
:104850000BF0230E0C6E02C10BF0A2EC0BF0240E39
:104860000C6E03C10BF0A2EC0BF000C15DF501C1B1
:104870005EF502C15FF503C160F54EEF24F004015F
:104880004C0E826F31EC0FF00401490E826F31EC57
:104890000FF004012C0E826F31EC0FF0250EB9ECF5
:1048A0000BF0E8CF00F1260EB9EC0BF0E8CF01F1E8
:1048B000270EB9EC0BF0E8CF02F1280EB9EC0BF0A3
:1048C000E8CF03F1FBEC33F0DEEC31F00401730EC2
:1048D000826F31EC0FF004012C0E826F31EC0FF07F
:1048E00058EC34F0290EB9EC0BF0E8CF00F1FBECFA
:1048F00033F0DEEC31F00401730E826F31EC0FF017
:1049000004012C0E826F31EC0FF057C500F158C531
:1049100001F159C502F15AC503F1FBEC33F0DEECAD
:1049200031F00401730E826F31EC0FF004012C0E94
:10493000826F31EC0FF058EC34F05CC500F1FBEC09
:1049400033F0DEEC31F004016D0E826F31EC0FF0CC
:1049500004012C0E826F31EC0FF05DC500F15EC5D5
:1049600001F15FC502F160C503F1C8EC2CF0040150
:104970002C0E826F31EC0FF03BEC0FF0ADEF2CF012
:1049800083C32AF184C32BF185C32CF186C32DF197
:1049900087C32EF188C32FF189C330F18AC331F167
:1049A0008BC332F18CC333F10101A6EC34F01DEC62
:1049B00034F0160E0C6E00C10BF0A2EC0BF0170ECB
:1049C0000C6E01C10BF0A2EC0BF0180E0C6E02C1C4
:1049D0000BF0A2EC0BF0190E0C6E03C10BF0A2EC65
:1049E0000BF000C18AF101C18BF102C18CF103C14E
:1049F0008DF100C18EF101C18FF102C190F103C1AF
:104A000091F1A2EF25F083C32AF184C32BF185C372
:104A10002CF186C32DF187C32EF188C32FF189C3F2
:104A200030F18AC331F18BC332F18CC333F1010110
:104A3000A6EC34F01DEC34F000C18AF101C18BF119
:104A400002C18CF103C18DF100C18EF101C18FF162
:104A500002C190F103C191F1A2EF25F083C32AF1C5
:104A600084C32BF185C32CF186C32DF187C32EF1AE
:104A700088C32FF189C330F18AC331F18CC332F17D
:104A80008DC333F10101A6EC34F01DEC34F00101CB
:104A9000000E046F000E056F010E066F000E076F0B
:104AA0006EEC33F01A0E0C6E00C10BF0A2EC0BF0A2
:104AB0001B0E0C6E01C10BF0A2EC0BF01C0E0C6E69
:104AC00002C10BF0A2EC0BF01D0E0C6E03C10BF03B
:104AD000A2EC0BF000C192F101C193F102C194F17B
:104AE00003C195F1A2EF25F083C32AF184C32BF112
:104AF00085C32CF186C32DF187C32EF188C32FF116
:104B000089C330F18AC331F18CC332F18DC333F1E3
:104B10000101A6EC34F01DEC34F00101000E046F2D
:104B2000000E056F010E066F000E076F6EEC33F07E
:104B300000C192F101C193F102C194F103C195F159
:104B4000A2EF25F0160EB9EC0BF0E8CF00F1170E2E
:104B5000B9EC0BF0E8CF01F1180EB9EC0BF0E8CF8F
:104B600002F1190EB9EC0BF0E8CF03F1FBEC33F0D6
:104B7000DEEC31F00401730E826F31EC0FF00401B2
:104B80002C0E826F31EC0FF08AC100F18BC101F164
:104B90008CC102F18DC103F1FBEC33F0DEEC31F09E
:104BA0000401730E826F31EC0FF004012C0E826F42
:104BB00031EC0FF01A0EB9EC0BF0E8CF00F11B0E40
:104BC000B9EC0BF0E8CF01F11C0EB9EC0BF0E8CF1B
:104BD00002F11D0EB9EC0BF0E8CF03F1C8EC2CF09C
:104BE00004012C0E826F31EC0FF092C100F193C1E1
:104BF00001F194C102F195C103F1C8EC2CF03BEC3A
:104C00000FF0ADEF2CF00401690E826F31EC0FF064
:104C100004012C0E826F31EC0FF00101040E006FC5
:104C2000000E016F000E026F000E036FFBEC33F0FD
:104C30002CC182F40401300E822731EC0FF02DC11B
:104C400082F40401300E822731EC0FF02EC182F481
:104C50000401300E822731EC0FF02FC182F40401E1
:104C6000300E822731EC0FF030C182F40401300E97
:104C7000822731EC0FF031C182F40401300E82271B
:104C800031EC0FF032C182F40401300E822731EC96
:104C90000FF033C182F40401300E822731EC0FF0A3
:104CA00004012C0E826F31EC0FF001010B0E006F2E
:104CB000000E016F000E026F000E036FFBEC33F06D
:104CC0002CC182F40401300E822731EC0FF02DC18B
:104CD00082F40401300E822731EC0FF02EC182F4F1
:104CE0000401300E822731EC0FF02FC182F4040151
:104CF000300E822731EC0FF030C182F40401300E07
:104D0000822731EC0FF031C182F40401300E82278A
:104D100031EC0FF032C182F40401300E822731EC05
:104D20000FF033C182F40401300E822731EC0FF012
:104D300004012C0E826F31EC0FF001012B0E006F7D
:104D4000000E016F000E026F000E036FFBEC33F0DC
:104D50002CC182F40401300E822731EC0FF02DC1FA
:104D600082F40401300E822731EC0FF02EC182F460
:104D70000401300E822731EC0FF02FC182F40401C0
:104D8000300E822731EC0FF030C182F40401300E76
:104D9000822731EC0FF031C182F40401300E8227FA
:104DA00031EC0FF032C182F40401300E822731EC75
:104DB0000FF033C182F40401300E822731EC0FF082
:104DC00004012C0E826F31EC0FF0200EF86EF76AA2
:104DD000F66A04010900F5CF82F431EC0FF0090006
:104DE000F5CF82F431EC0FF00900F5CF82F431EC0D
:104DF0000FF00900F5CF82F431EC0FF00900F5CF88
:104E000082F431EC0FF00900F5CF82F431EC0FF0B1
:104E10000900F5CF82F431EC0FF00900F5CF82F4F0
:104E200031EC0FF03BEC0FF0ADEF2CF08351630A47
:104E3000D8A4ADEF2CF08451610AD8A4ADEF2CF0CA
:104E400085516C0AD8A4ADEF2CF08651410A3FE0A1
:104E50008651440A1BE08651420AD8B47AEF27F003
:104E60008651350AD8B437EF2EF08651360AD8B4B9
:104E70008CEF2EF08651370AD8B4F5EF2EF086511C
:104E8000380AD8B453EF2FF0ADEF2CF00798079AFB
:104E900004017A0E826F31EC0FF00401780E826FFC
:104EA00031EC0FF00401640E826F31EC0FF004015D
:104EB000550E826F31EC0FF063EF27F004014C0EBA
:104EC000826F31EC0FF03BEC0FF0ADEF2CF0078868
:104ED000079A04017A0E826F31EC0FF00401410E43
:104EE000826F31EC0FF00401610E826F31EC0FF034
:104EF00057EF27F00798078A04017A0E826F31EC8A
:104F00000FF00401420E826F31EC0FF00401610ECC
:104F1000826F31EC0FF057EF27F00101666798EFD1
:104F200027F0676798EF27F0686798EF27F06967C1
:104F300015D04F67A3EF27F05067A3EF27F0516715
:104F4000A3EF27F052670AD00101000E006F000E98
:104F5000016F000E026F000E036F120011B80AD02D
:104F60000101620E046F010E056F000E066F000E48
:104F7000076F09D00101A70E046F020E056F000E26
:104F8000066F000E076F66C100F167C101F168C1CD
:104F900002F169C103F15DEC33F003BF40EF28F08B
:104FA000119A119C0101000E046FA80E056F550E99
:104FB000066F020E076F66C100F167C101F168C19B
:104FC00002F169C103F166C186F167C187F168C169
:104FD00088F169C189F15DEC33F003BF0BD00101A9
:104FE000000E866FA80E876F550E886F020E896FB0
:104FF000118A119C0E0EB9EC0BF0E8CF18F10F0ED0
:10500000B9EC0BF0E8CF19F1100EB9EC0BF0E8CFCA
:105010001AF1110EB9EC0BF0E8CF1BF1A6EC32F04F
:1050200086C104F187C105F188C106F189C107F184
:105030005DEC33F007826AEC32F0A6EC32F00792B6
:105040006AEC32F086C100F187C101F188C102F13A
:1050500089C103F107926AEC32F0CC0E046FE00EC6
:10506000056F870E066F050E076F5DEC33F000C10C
:1050700018F101C119F102C11AF103C11BF13BD0B2
:10508000119C119A0101800E006F1A0E016F060E1D
:10509000026F000E036F4FC104F150C105F151C101
:1050A00006F152C107F15DEC33F003AF05D058ECC7
:1050B00034F0118C119A12000E0EB9EC0BF0E8CFFF
:1050C00018F10F0EB9EC0BF0E8CF19F1100EB9EC96
:1050D0000BF0E8CF1AF1110EB9EC0BF0E8CF1BF191
:1050E0004FC100F150C101F151C102F152C103F1B0
:1050F00007826AEC32F018C100F119C101F11AC13E
:1051000002F11BC103F112000401730E826F31EC36
:105110000FF004012C0E826F31EC0FF0078462C196
:1051200066F163C167F164C168F165C169F14BC1A2
:105130004FF14CC150F14DC151F14EC152F157C127
:1051400059F158C15AF10794AAEC28F03BEC0FF042
:10515000ADEF2CF066C100F167C101F168C102F149
:1051600069C103F10101FBEC33F0DEEC31F0040125
:10517000630E826F31EC0FF004012C0E826F31EC64
:105180000FF04FC100F150C101F151C102F152C104
:1051900003F10101FBEC33F0DEEC31F00401660EAB
:1051A000826F31EC0FF004012C0E826F31EC0FF0A6
:1051B00058EC34F059C100F15AC101F10101FBEC86
:1051C00033F0DEEC31F00401740E826F31EC0FF03D
:1051D000120010820401530E826F31EC0FF00401B3
:1051E0002C0E826F31EC0FF083C32AF184C32BF1B4
:1051F00085C32CF186C32DF187C32EF188C32FF10F
:1052000089C330F18AC331F18BC332F18CC333F1DE
:105210000101A6EC34F01DEC34F000C166F101C1CF
:1052200067F102C168F103C169F18EC32AF18FC32E
:105230002BF190C32CF191C32DF192C32EF193C3A6
:105240002FF194C330F195C331F196C332F197C376
:1052500033F10101A6EC34F01DEC34F000C14FF144
:1052600001C150F102C151F103C152F199EC34F086
:1052700099C32FF19AC330F19BC331F19CC332F132
:105280009DC333F10101A6EC34F01DEC34F000C1F4
:1052900059F101C15AF1AAEC28F004012C0E826FD9
:1052A00031EC0FF05DEF29F018A001D0108C825185
:1052B000520A02E10F8201D00F928251750A02E177
:1052C000108401D010948251550A02E1108601D059
:1052D000109611A003D011A401D01084078410B23D
:1052E000CBEF29F010A4B7EF29F0B6C166F1B7C132
:1052F00067F1B8C168F1B9C169F1BAC16AF1BBC15E
:105300006BF1BCC16CF1BDC16DF1BEC16EF1BFC12D
:105310006FF1C0C170F1C1C171F1C2C172F1C3C1FD
:1053200073F1C4C174F1C5C175F1C6C176F1C7C1CD
:1053300077F1C8C178F1C9C179F1CAC17AF1CBC19D
:105340007BF1CCC17CF1CDC17DF1CEC17EF1CFC16D
:105350007FF1D0C180F1D1C181F1D2C182F1D3C13D
:1053600083F1D4C184F1D5C185F1BFEF29F062C1C9
:1053700066F163C167F164C168F165C169F14BC150
:105380004FF14CC150F14DC151F14EC152F157C1D5
:1053900059F158C15AF107940FA0EDEF29F001011E
:1053A0009267DAEF29F09367DAEF29F09467DAEF82
:1053B00029F09567DEEF29F0EDEF29F08DEC27F06D
:1053C00092C104F193C105F194C106F195C107F1B1
:1053D0005DEC33F003BF73EF2CF08DEC27F001018F
:1053E000000E046F000E056F010E066F000E076FB2
:1053F0008EEC33F011A02CD011A22AD0FBEC33F0AC
:10540000296701D007D004012D0E826F31EC0FF017
:1054100071EF2CF030C182F40401300E822731ECA0
:105420000FF031C182F40401300E822731EC0FF00D
:1054300032C182F40401300E822731EC0FF033C107
:1054400082F40401300E822731EC0FF071EF2CF062
:1054500012A8C5D0129819C01AF01A3A1A42070EAB
:105460001A1600011A50000AD8B4BBEF2AF0000146
:105470001A50010AD8B447EF2AF000011A50020A64
:10548000D8B445EF2AF0EDEF2AF0EDEF2AF058EC12
:1054900034F029C001F12AC000F1D8900133003363
:1054A000D890013300330101630E046F000E056FC5
:1054B000000E066F000E076F8EEC33F0280E046F9F
:1054C000000E056F000E066F000E076F5DEC33F0E7
:1054D00000C12CF058EC34F027C001F1019F019D70
:1054E00028C000F10101A40E046F000E056F000E2C
:1054F000066F000E076F8EEC33F000C12BF000C179
:1055000004F101C105F102C106F103C107F1640E06
:10551000006F000E016F000E026F000E036F5DEC56
:1055200033F0050E046F000E056F000E066F000EBF
:10553000076F8EEC33F000C104F101C105F102C127
:1055400006F103C107F158EC34F02CC000F15DEC1A
:1055500033F000C12DF02DC0E8FF050F2C5C03E7F0
:105560008A84EDEF2AF02DC0E8FF0A0F2C5C01E6DB
:105570008A94EDEF2AF000C124F101C125F102C1A6
:1055800026F103C127F158EC34F05EEC34F01950E9
:105590001F0BE8CF00F10101640E046F000E056FD0
:1055A000000E066F000E076F6EEC33F024C104F19D
:1055B00025C105F126C106F127C107F15DEC33F0E5
:1055C00003BF02D08A9401D08A8424C100F125C18E
:1055D00001F126C102F127C103F173EF2CF010AEE7
:1055E0004BD0109E00C108F101C109F102C10AF1BE
:1055F00003C10BF1FBEC33F030C1D6F131C1D7F16F
:1056000032C1D8F133C1D9F108C100F109C101F1AA
:105610000AC102F10BC103F101016C0E046F070E08
:10562000056F000E066F000E076F5DEC33F003BFD1
:1056300004D00101550EDA6F1CD008C100F109C178
:1056400001F10AC102F10BC103F10101A40E046FC3
:10565000060E056F000E066F000E076F5DEC33F04F
:1056600003BF04D001017F0EDA6F03D00101FF0EEA
:10567000DA6F1B8E73EF2CF010A446EF2BF00401B1
:10568000750E826F31EC0FF04BEF2BF00401720EB0
:10569000826F31EC0FF004012C0E826F31EC0FF0B1
:1056A000FBEC33F029675AEF2BF00401200E826FD8
:1056B0005DEF2BF004012D0E826F31EC0FF030C145
:1056C00082F40401300E822731EC0FF031C182F4F4
:1056D0000401300E822731EC0FF004012E0E826F90
:1056E00031EC0FF032C182F40401300E822731EC2C
:1056F0000FF033C182F40401300E822731EC0FF039
:1057000004016D0E826F31EC0FF004012C0E826FDC
:1057100031EC0FF04FC100F150C101F151C102F164
:1057200052C103F10101FBEC33F0DEEC31F0040176
:10573000480E826F31EC0FF004017A0E826F31EC6B
:105740000FF004012C0E826F31EC0FF066C100F1F6
:1057500067C101F168C102F169C103F10101FBEC0C
:1057600033F0DEEC31F00401630E826F31EC0FF0A8
:1057700004012C0E826F31EC0FF066C100F167C19D
:1057800001F168C102F169C103F101010A0E046F60
:10579000000E056F000E066F000E076F6EEC33F003
:1057A000000E046F120E056F000E066F000E076FDD
:1057B0008EEC33F0FBEC33F02AC182F40401300E9E
:1057C000822731EC0FF02BC182F40401300E8227C6
:1057D00031EC0FF02CC182F40401300E822731EC41
:1057E0000FF02DC182F40401300E822731EC0FF04E
:1057F0002EC182F40401300E822731EC0FF02FC14C
:1058000082F40401300E822731EC0FF030C182F4B3
:105810000401300E822731EC0FF004012E0E826F4E
:1058200031EC0FF031C182F40401300E822731ECEB
:105830000FF032C182F40401300E822731EC0FF0F8
:1058400033C182F40401300E822731EC0FF00401E1
:10585000730E826F31EC0FF004012C0E826F31EC6D
:105860000FF058EC34F059C100F15AC101F1D7ECF6
:105870002DF00FB23FEF2CF00FA071EF2CF00401D0
:105880002C0E826F31EC0FF0200EF86EF76AF66A7C
:1058900004010900F5CF82F431EC0FF00900F5CFD7
:1058A00082F431EC0FF00900F5CF82F431EC0FF007
:1058B0000900F5CF82F431EC0FF00900F5CF82F446
:1058C00031EC0FF00900F5CF82F431EC0FF0090054
:1058D000F5CF82F431EC0FF00900F5CF82F431EC12
:1058E0000FF03BEC0FF00F90ADEF2CF00401630EC6
:1058F000826F31EC0FF004012C0E826F31EC0FF04F
:10590000B3EC2CF004012C0E826F31EC0FF026EC7E
:105910002DF004012C0E826F31EC0FF0A2EC2DF073
:1059200004012C0E826F31EC0FF00101F80E006FB4
:10593000CD0E016F660E026F030E036FC8EC2CF0E4
:1059400004012C0E826F31EC0FF0B8EC2DF03BEC23
:105950000FF0ADEF2CF03BEC0FF00301C26B0790A2
:105960001092BCEF2FF0D8900E0EB9EC0BF0E8CFF0
:1059700000F10F0EB9EC0BF0E8CF01F1100EB9EC0D
:105980000BF0E8CF02F1110EB9EC0BF0E8CF03F108
:105990000101000E046F000E056F010E066F000E70
:1059A000076F8EEC33F0FBEC33F02AC182F4040174
:1059B000300E822731EC0FF02BC182F40401300E3F
:1059C000822731EC0FF02CC182F40401300E8227C3
:1059D00031EC0FF02DC182F40401300E822731EC3E
:1059E0000FF02EC182F40401300E822731EC0FF04B
:1059F0002FC182F40401300E822731EC0FF030C148
:105A000082F40401300E822731EC0FF031C182F4B0
:105A10000401300E822731EC0FF004012E0E826F4C
:105A200031EC0FF032C182F40401300E822731ECE8
:105A30000FF033C182F40401300E822731EC0FF0F5
:105A400004016D0E826F31EC0FF01200120EB9ECF2
:105A50000BF0E8CF00F1130EB9EC0BF0E8CF01F139
:105A6000140EB9EC0BF0E8CF02F1150EB9EC0BF007
:105A7000E8CF03F101010A0E046F000E056F000E5E
:105A8000066F000E076F6EEC33F0000E046F120EFF
:105A9000056F000E066F000E076F8EEC33F0FBEC07
:105AA00033F02AC182F40401300E822731EC0FF06A
:105AB0002BC182F40401300E822731EC0FF02CC18F
:105AC00082F40401300E822731EC0FF02DC182F4F4
:105AD0000401300E822731EC0FF02EC182F4040154
:105AE000300E822731EC0FF02FC182F40401300E0A
:105AF000822731EC0FF030C182F40401300E82278E
:105B000031EC0FF004012E0E826F31EC0FF031C139
:105B100082F40401300E822731EC0FF032C182F49E
:105B20000401300E822731EC0FF033C182F40401FE
:105B3000300E822731EC0FF00401730E826F31ECCE
:105B40000FF012000A0EB9EC0BF0E8CF00F10B0ECB
:105B5000B9EC0BF0E8CF01F10C0EB9EC0BF0E8CF8B
:105B600002F10D0EB9EC0BF0E8CF03F1D7EF2DF0F9
:105B7000060EB9EC0BF0E8CF00F1070EB9EC0BF014
:105B8000E8CF01F1080EB9EC0BF0E8CF02F1090EF5
:105B9000B9EC0BF0E8CF03F1D7EF2DF0010158EC91
:105BA00034F0078457C100F158C101F10794010195
:105BB000E80E046F800E056F000E066F000E076F73
:105BC0006EEC33F0000E046F040E056F000E066FCE
:105BD000000E076F8EEC33F0880E046F130E056F06
:105BE000000E066F000E076F5DEC33F00A0E046FB7
:105BF000000E056F000E066F000E076F8EEC33F07F
:105C0000FBEC33F0010129670BEF2EF00401200EAD
:105C1000826F0EEF2EF004012D0E826F31EC0FF02B
:105C200030C182F40401300E822731EC0FF031C113
:105C300082F40401300E822731EC0FF032C182F47D
:105C40000401300E822731EC0FF004012E0E826F1A
:105C500031EC0FF033C182F40401300E822731ECB5
:105C60000FF00401430E826F31EC0FF0120087C376
:105C70002AF188C32BF189C32CF18AC32DF18BC380
:105C80002EF18CC32FF18DC330F18EC331F190C34F
:105C900032F191C333F10101296BA6EC34F01DEC14
:105CA00034F00101000E046F000E056F010E066F47
:105CB000000E076F6EEC33F00E0E0C6E00C10BF091
:105CC000A2EC0BF00F0E0C6E01C10BF0A2EC0BF06E
:105CD000100E0C6E02C10BF0A2EC0BF0110E0C6E4C
:105CE00003C10BF0A2EC0BF004017A0E826F31ECD1
:105CF0000FF004012C0E826F31EC0FF00401350E11
:105D0000826F31EC0FF004012C0E826F31EC0FF03A
:105D1000B3EC2CF063EF27F087C32AF188C32BF193
:105D200089C32CF18AC32DF18BC32EF18CC32FF1C3
:105D30008DC330F18EC331F190C332F191C333F191
:105D40000101296BA6EC34F01DEC34F0880E046FD1
:105D5000130E056F000E066F000E076F62EC33F036
:105D6000000E046F040E056F000E066F000E076F25
:105D70006EEC33F00101E80E046F800E056F000E2B
:105D8000066F000E076F8EEC33F00A0E0C6E00C12A
:105D90000BF0A2EC0BF00B0E0C6E01C10BF0A2ECA1
:105DA0000BF00C0E0C6E02C10BF0A2EC0BF00D0E02
:105DB0000C6E03C10BF0A2EC0BF004017A0E826FA3
:105DC00031EC0FF004012C0E826F31EC0FF0040166
:105DD000360E826F31EC0FF004012C0E826F31EC25
:105DE0000FF0A2EC2DF063EF27F087C32AF188C3F0
:105DF0002BF189C32CF18AC32DF18BC32EF18CC3F7
:105E00002FF18DC330F18FC331F190C332F191C3C3
:105E100033F10101A6EC34F01DEC34F0000E046FF8
:105E2000120E056F000E066F000E076F6EEC33F05A
:105E300001010A0E046F000E056F000E066F000EC2
:105E4000076F8EEC33F0120E0C6E00C10BF0A2EC5B
:105E50000BF0130E0C6E01C10BF0A2EC0BF0140E44
:105E60000C6E02C10BF0A2EC0BF0150E0C6E03C110
:105E70000BF0A2EC0BF004017A0E826F31EC0FF004
:105E800004012C0E826F31EC0FF00401370E826F8B
:105E900031EC0FF004012C0E826F31EC0FF026EC88
:105EA0002DF063EF27F087C32AF188C32BF189C354
:105EB0002CF18AC32DF18BC32EF18CC32FF18DC32E
:105EC00030F18EC331F190C332F191C333F101014E
:105ED000296BA6EC34F01DEC34F0880E046F130E21
:105EE000056F000E066F000E076F62EC33F0000EB8
:105EF000046F040E056F000E066F000E076F6EEC48
:105F000033F00101E80E046F800E056F000E066F7E
:105F1000000E076F8EEC33F0060E0C6E00C10BF016
:105F2000A2EC0BF0070E0C6E01C10BF0A2EC0BF013
:105F3000080E0C6E02C10BF0A2EC0BF0090E0C6EF9
:105F400003C10BF0A2EC0BF004017A0E826F31EC6E
:105F50000FF004012C0E826F31EC0FF00401380EAB
:105F6000826F31EC0FF004012C0E826F31EC0FF0D8
:105F7000B8EC2DF063EF27F007A830EF30F0010107
:105F8000800E006F1A0E016F060E026F000E036F77
:105F90004BC104F14CC105F14DC106F14EC107F1F1
:105FA0005DEC33F003BF77EF30F0D8EC31F04BC14C
:105FB00000F14CC101F14DC102F14EC103F1078264
:105FC0006AEC32F018C104F119C105F11AC106F1E9
:105FD0001BC107F1F80E006FCD0E016F660E026F48
:105FE000030E036F5DEC33F00E0E0C6E00C10BF070
:105FF000A2EC0BF00F0E0C6E01C10BF0A2EC0BF03B
:10600000100E0C6E02C10BF0A2EC0BF0110E0C6E18
:1060100003C10BF0A2EC0BF00784010158EC34F043
:1060200057C100F158C101F107940A0E0C6E00C16E
:106030000BF0A2EC0BF00B0E0C6E01C10BF0A2ECFE
:106040000BF00C0E0C6E02C10BF0A2EC0BF00D0E5F
:106050000C6E03C10BF0A2EC0BF0079877EF30F059
:1060600007AA77EF30F00784010158EC34F057C1EC
:1060700000F158C101F10794060E0C6E00C10BF03F
:10608000A2EC0BF0070E0C6E01C10BF0A2EC0BF0B2
:10609000080E0C6E02C10BF0A2EC0BF0090E0C6E98
:1060A00003C10BF0A2EC0BF0078462C100F163C1E5
:1060B00001F164C102F165C103F10794120E0C6E87
:1060C00000C10BF0A2EC0BF0130E0C6E01C10BF033
:1060D000A2EC0BF0140E0C6E02C10BF0A2EC0BF054
:1060E000150E0C6E03C10BF0A2EC0BF0079A040125
:1060F000805181197F0B0BE09EA809D014EE00F0AF
:1061000081517F0BE126E750812B0F01AD6E050118
:106110002F51010A13E081AA9EEF30F005012F51A3
:10612000000A0AE00FB89EEF30F0050130679EEFDD
:1061300030F00FB89EEF30F015EF3EF081B8B3EFBE
:1061400030F0A7EC36F005012F51020A02E0B3EF60
:1061500030F05C2FB3EF30F05BC55CF50501010E4C
:10616000306F3C0E316F80EF0EF006013251385D1A
:106170003351D8A0010F395D800BD8A4C4EF30F0A3
:1061800032C638F633C639F6120006013251365D92
:106190003351D8A0010F375D800BD8B4D4EF30F065
:1061A00032C636F633C637F6120007841AC632F600
:1061B0001BC633F61CC638F61DC639F6B5EC30F0F2
:1061C0001EC632F61FC633F6B5EC30F020C632F6E6
:1061D00021C633F6B5EC30F01AC632F61BC633F6DC
:1061E0001CC636F61DC637F6C5EC30F01EC632F6B4
:1061F0001FC633F6C5EC30F020C632F621C633F6A2
:10620000C5EC30F03851365F3951D8A03929375FA5
:1062100058EC34F036C600F137C601F164EC34F0C6
:1062200000C13AF601C13BF622C632F623C633F668
:1062300024C638F625C639F6B5EC30F026C632F657
:1062400027C633F6B5EC30F028C632F629C633F649
:10625000B5EC30F022C632F623C633F624C636F645
:1062600025C637F6C5EC30F026C632F627C633F61B
:10627000C5EC30F028C632F629C633F6C5EC30F04E
:106280003851365F3951D8A03929375F58EC34F08E
:1062900036C600F137C601F164EC34F000C13CF6BB
:1062A00001C13DF62AC632F62BC633F62CC638F6A7
:1062B0002DC639F6B5EC30F02EC632F62FC633F6C1
:1062C000B5EC30F030C632F631C633F6B5EC30F00E
:1062D0002AC632F62BC633F62CC636F62DC637F64E
:1062E000C5EC30F02EC632F62FC633F6C5EC30F0D2
:1062F00030C632F631C633F6C5EC30F03851365F71
:106300003951D8A03929375F58EC34F036C600F13E
:1063100037C601F164EC34F000C13EF601C13FF62E
:106320003AC632F63BC633F63CC636F63DC637F6BD
:10633000C5EC30F03EC632F63FC633F6C5EC30F061
:106340000794120018C100F119C101F11AC102F13C
:106350001BC103F1000E046F000E056F010E066FE6
:10636000000E076F8EEC33F029A1CDEF31F02051F4
:10637000D8B4CDEF31F018C100F119C101F11AC143
:1063800002F11BC103F1000E046F000E056F0A0E2F
:10639000066F000E076F8EEC33F0120001010451FE
:1063A0000013055101130651021307510313120084
:1063B0000101186B196B1A6B1B6B12002AC182F456
:1063C0000401300E822731EC0FF02BC182F404015E
:1063D000300E822731EC0FF02CC182F40401300E14
:1063E000822731EC0FF02DC182F40401300E822798
:1063F00031EC0FF02EC182F40401300E822731EC13
:106400000FF02FC182F40401300E822731EC0FF01F
:1064100030C182F40401300E822731EC0FF031C11B
:1064200082F40401300E822731EC0FF032C182F485
:106430000401300E822731EC0FF033C182F40401E5
:10644000300E822731EC0FF012002FC182F40401CC
:10645000300E822731EC0FF030C182F40401300E8F
:10646000822731EC0FF031C182F40401300E822713
:1064700031EC0FF032C182F40401300E822731EC8E
:106480000FF033C182F40401300E822731EC0FF09B
:106490001200060E1D6E060E1E6E060E1F6E1D2EBF
:1064A0004FEF32F01E2E4FEF32F01F2E4FEF32F033
:1064B0008B84020E1D6E020E1E6E020E1F6E1D2EAE
:1064C0005FEF32F01E2E5FEF32F01F2E5FEF32F0E3
:1064D0008B9412000101005305E1015303E10253C3
:1064E00001E1002B2DEC33F058EC34F03951006F02
:1064F0003A51016F420E046F4B0E056F000E066F8E
:10650000000E076F6EEC33F000C104F101C105F11C
:1065100002C106F103C107F118C100F119C101F16F
:106520001AC102F11BC103F107B29BEF32F062EC1A
:1065300033F09DEF32F05DEC33F000C118F101C192
:1065400019F102C11AF103C11BF1120058EC34F029
:1065500059C100F15AC101F1060EB9EC0BF0E8CFB8
:1065600004F1070EB9EC0BF0E8CF05F1080EB9EC19
:106570000BF0E8CF06F1090EB9EC0BF0E8CF07F10C
:106580005DEC33F000C124F101C125F102C126F117
:1065900003C127F1290E046F000E056F000E066F70
:1065A000000E076F6EEC33F0EE0E046F430E056FB6
:1065B000000E066F000E076F62EC33F024C104F189
:1065C00025C105F126C106F127C107F16EEC33F0B4
:1065D00000C11CF101C11DF102C11EF103C11FF177
:1065E000120EB9EC0BF0E8CF04F1130EB9EC0BF07E
:1065F000E8CF05F1140EB9EC0BF0E8CF06F1150E5B
:10660000B9EC0BF0E8CF07F10D0E006F000E016F33
:10661000000E026F000E036F6EEC33F0180E046F65
:10662000000E056F000E066F000E076F8EEC33F044
:106630001CC104F11DC105F11EC106F11FC107F106
:1066400062EC33F06A0E046F2A0E056F000E066FBF
:10665000000E076F5DEC33F01200BF0EFA6E200ED5
:106660003A6F396BD8900037013702370337D8B00B
:106670003EEF33F03A2F33EF33F039073A07035345
:10668000D8B412000331070B80093F6F03390F0B99
:10669000010F396F80EC5FF0406F390580EC5FF0DF
:1066A000405D405F396B3F33D8B0392739333FA95C
:1066B00053EF33F040513927120001017DEC34F0E3
:1066C000D8B01200010103510719346F40EC34F0C7
:1066D000D8900751031934AF800F12000101346BB9
:1066E00064EC34F0D8A07AEC34F0D8B012004FEC5F
:1066F00034F058EC34F01F0E366F90EC34F00B355C
:10670000D8B040EC34F0D8A00335D8B01200362F02
:106710007DEF33F034B167EC34F012000101346BDB
:1067200004510511061107110008D8A064EC34F0DB
:10673000D8A07AEC34F0D8B01200086B096B0A6B61
:106740000B6B90EC34F01F0E366F90EC34F0075169
:106750000B5DD8A4B8EF33F006510A5DD8A4B8EFAA
:1067600033F00551095DD8A4B8EF33F00451085D4A
:10677000D8A0CBEF33F00451085F0551D8A0053DF8
:10678000095F0651D8A0063D0A5F0751D8A0073D12
:106790000B5FD8900081362FA5EF33F034B167EC52
:1067A00034F0346B64EC34F0D89094EC34F007514E
:1067B0000B5DD8A4E8EF33F006510A5DD8A4E8EFEA
:1067C00033F00551095DD8A4E8EF33F00451085DBA
:1067D000D8A0F7EF33F0003FF7EF33F0013FF7EFCA
:1067E00033F0023FF7EF33F0032BD8B4120034B18B
:1067F00067EC34F012000101346B64EC34F0D8B073
:10680000120099EC34F0200E366F00370137023752
:10681000033711EE33F00A0E376FE7360A0EE75CE6
:10682000D8B0E76EE552372F0DEF34F0362F05EF75
:1068300034F034B12981D890120001010A0E346F6E
:10684000200E366F11EE29F03451376F0A0ED890B2
:10685000E652D8B0E726E732372F28EF34F003337B
:10686000023301330033362F22EF34F0E750FF0FAD
:10687000D8A00335D8B0120029B167EC34F012006B
:10688000045100270551D8B0053D01270651D8B065
:10689000063D02270751D8B0073D032712000051DB
:1068A000086F0151096F02510A6F03510B6F1200FB
:1068B0000101006B016B026B036B12000101046BA1
:1068C000056B066B076B12000335D8A0120003514D
:1068D000800B001F011F021F031F003F77EF34F0E2
:1068E000013F77EF34F0023F77EF34F0032B342B86
:1068F000032512000735D8A012000751800B041F92
:10690000051F061F071F043F8DEF34F0053F8DEF75
:1069100034F0063F8DEF34F0072B342B072512009F
:106920000037013702370337083709370A370B3783
:1069300012000101296B2A6B2B6B2C6B2D6B2E6BBC
:106940002F6B306B316B326B336B120001012A51AC
:106950000F0B2A6F2B510F0B2B6F2C510F0B2C6F22
:106960002D510F0B2D6F2E510F0B2E6F2F510F0B23
:106970002F6F30510F0B306F31510F0B316F325180
:106980000F0B326F33510F0B336F1200899C000EC7
:10699000C76E200EC66E9E96C69EC50EC96EFF0EB1
:1069A0009EB602D0E82EFCD79E96C69E000EC96EFB
:1069B000FF0E9EB602D0E82EFCD7C9CF00F69E96F9
:1069C000C69E000EC96EFF0E9EB602D0E82EFCD702
:1069D000C9CF01F6898C1200000EC76E200EC66E5C
:1069E000899C9E96C69EC80EC96EFF0E9EB602D0AA
:1069F000E82EFCD79E96C69E000EC96EFF0E9EB670
:106A000002D0E82EFCD7C9CF02F69E96C69E000E95
:106A1000C96EFF0E9EB602D0E82EFCD7C9CF03F692
:106A20009E96C69E000EC96EFF0E9EB602D0E82E40
:106A3000FCD7C9CF0AF69E96C69E000EC96EFF0E01
:106A40009EB602D0E82EFCD7C9CF0BF69E96C69E06
:106A5000000EC96EFF0E9EB602D0E82EFCD7C9CF3D
:106A600012F69E96C69E000EC96EFF0E9EB602D00E
:106A7000E82EFCD7C9CF13F6898C1200000EC76E22
:106A8000200EC66E899C9E96C69EE80EC96EFF0EAD
:106A90009EB602D0E82EFCD79E96C69E000EC96E0A
:106AA000FF0E9EB602D0E82EFCD7C9CF1AF69E96EE
:106AB000C69E000EC96EFF0E9EB602D0E82EFCD711
:106AC000C9CF1BF69E96C69E000EC96EFF0E9EB6DF
:106AD00002D0E82EFCD7C9CF22F69E96C69E000EA5
:106AE000C96EFF0E9EB602D0E82EFCD7C9CF23F6A2
:106AF0009E96C69E000EC96EFF0E9EB602D0E82E70
:106B0000FCD7C9CF2AF69E96C69E000EC96EFF0E10
:106B10009EB602D0E82EFCD7C9CF2BF6898C120086
:106B2000000EC76E200EC66E899C9E96C69E240ED1
:106B3000C96EFF0E9EB602D0E82EFCD79E96C69E6A
:106B4000E40EC96EFF0E9EB602D0E82EFCD7898CEB
:106B5000899C9E96C69E200EC96EFF0E9EB602D0E0
:106B6000E82EFCD79E96C69E5F0EC96EFF0E9EB69F
:106B700002D0E82EFCD7898C899C9E96C69E210E59
:106B8000C96EFF0E9EB602D0E82EFCD79E96C69E1A
:106B9000C00EC96EFF0E9EB602D0E82EFCD7898CBF
:106BA000899C9E96C69E260EC96EFF0E9EB602D08A
:106BB000E82EFCD79E96C69E000EC96EFF0E9EB6AE
:106BC00002D0E82EFCD7898C120010A806D0899438
:106BD000000EC76E220EC66E05D08984000EC76EE9
:106BE000220EC66E050EE82EFED7120010A802D0A7
:106BF000898401D08994050EE82EFED71200E5ECB9
:106C000035F09E96C69E000EC96EFF0E9EB602D04F
:106C1000E82EFCD79E96C69E000EC96EFF0E9EB64D
:106C200002D0E82EFCD7C9CFABF59E96C69E000ECB
:106C3000C96EFF0E9EB602D0E82EFCD7C9CFACF5C8
:106C40009E96C69E000EC96EFF0E9EB602D0E82E1E
:106C5000FCD7C9CFADF59E96C69E000EC96EFF0E3D
:106C60009EB602D0E82EFCD7C9CFAEF59E96C69E42
:106C7000000EC96EFF0E9EB602D0E82EFCD7C9CF1B
:106C8000AFF59E96C69E000EC96EFF0E9EB602D050
:106C9000E82EFCD7C9CFB0F59E96C69E000EC96EF1
:106CA000FF0E9EB602D0E82EFCD7C9CFB1F5F6ECA8
:106CB00035F01200E5EC35F09E96C69E800EC96E4A
:106CC000FF0E9EB602D0E82EFCD79E96C69EABC5A0
:106CD000C9FFFF0E9EB602D0E82EFCD79E96C69E38
:106CE000ACC5C9FFFF0E9EB602D0E82EFCD79E961B
:106CF000C69EADC5C9FFFF0E9EB602D0E82EFCD7DA
:106D00009E96C69EAEC5C9FFFF0E9EB602D0E82E67
:106D1000FCD79E96C69EAFC5C9FFFF0E9EB602D099
:106D2000E82EFCD79E96C69EB0C5C9FFFF0E9EB644
:106D300002D0E82EFCD79E96C69EB1C5C9FFFF0EB5
:106D40009EB602D0E82EFCD7F6EC35F01200E5EC4A
:106D500035F09E96C69E070EC96EFF0E9EB602D0F7
:106D6000E82EFCD79E96C69E000EC96EFF0E9EB6FC
:106D700002D0E82EFCD7C9CFABF59E96C69E000E7A
:106D8000C96EFF0E9EB602D0E82EFCD7C9CFACF577
:106D90009E96C69E000EC96EFF0E9EB602D0E82ECD
:106DA000FCD7C9CFADF59E96C69E000EC96EFF0EEC
:106DB0009EB602D0E82EFCD7C9CFAEF5F6EC35F082
:106DC000E5EC35F09E96C69E21C0C9FFFF0E9EB62B
:106DD00002D0E82EFCD79E96C69E000EC96EFF0E0E
:106DE0009EB602D0E82EFCD7C9CFB2F5F6EC35F04E
:106DF0001200E5EC35F09E96C69E870EC96EFF0E1A
:106E00009EB602D0E82EFCD79E96C69EABC5C9FFA3
:106E1000FF0E9EB602D0E82EFCD79E96C69EACC54D
:106E2000C9FFFF0E9EB602D0E82EFCD79E96C69EE6
:106E3000ADC5C9FFFF0E9EB602D0E82EFCD79E96C8
:106E4000C69EAEC5C9FFFF0E9EB602D0E82EFCD787
:106E5000F6EC35F0E5EC35F09E96C69E22C0C9FFF3
:106E6000FF0E9EB602D0E82EFCD79E96C69EB2C5F7
:106E7000C9FFFF0E9EB602D0E82EFCD7F6EC35F027
:106E80001200E5EC35F09E96C69E870EC96EFF0E89
:106E90009EB602D0E82EFCD79E96C69E000EC96E06
:106EA000FF0E9EB602D0E82EFCD79E96C69E800EA0
:106EB000C96EFF0E9EB602D0E82EFCD79E96C69EE7
:106EC000800EC96EFF0E9EB602D0E82EFCD79E96AD
:106ED000C69E800EC96EFF0E9EB602D0E82EFCD76D
:106EE000F6EC35F01200E5EC35F09E96C69E870E66
:106EF000C96EFF0E9EB602D0E82EFCD79E96C69EA7
:106F0000000EC96EFF0E9EB602D0E82EFCD79E96EC
:106F1000C69E000EC96EFF0E9EB602D0E82EFCD7AC
:106F20009E96C69E800EC96EFF0E9EB602D0E82EBB
:106F3000FCD79E96C69E800EC96EFF0E9EB602D0EE
:106F4000E82EFCD7F6EC35F0120010A82DD0E5ECB9
:106F500035F09E96C69E22C0C9FFFF0E9EB602D097
:106F6000E82EFCD79E96C69E450EC96EFF0E9EB6B5
:106F700002D0E82EFCD7F6EC35F0E5EC35F09E9625
:106F8000C69E8F0EC96EFF0E9EB602D0E82EFCD7AD
:106F90009E96C69E000EC96EFF0E9EB602D0E82ECB
:106FA000FCD7F6EC35F01200E5EC35F09E96C69E67
:106FB00022C0C9FFFF0E9EB602D0E82EFCD79E96D7
:106FC000C69E010EC96EFF0E9EB602D0E82EFCD7FB
:106FD000F6EC35F0E5EC35F09E96C69E910EC96E46
:106FE000FF0E9EB602D0E82EFCD79E96C69EA50E3A
:106FF000C96EFF0E9EB602D0E82EFCD7F6EC35F037
:107000001200E5EC35F09E96C69E22C0C9FFFF0E29
:107010009EB602D0E82EFCD79E96C69E810EC96E03
:10702000FF0E9EB602D0E82EFCD7F6EC35F012002B
:10703000E5EC35F09E96C69E22C0C9FFFF0E9EB6B7
:1070400002D0E82EFCD79E96C69E010EC96EFF0E9A
:107050009EB602D0E82EFCD7F6EC35F01200E5EC37
:1070600035F09E96C69E910EC96EFF0E9EB602D05A
:10707000E82EFCD79E96C69EA50EC96EFF0E9EB644
:1070800002D0E82EFCD7F6EC35F01200E5EC35F036
:107090009E96C69E910EC96EFF0E9EB602D0E82E39
:1070A000FCD79E96C69E000EC96EFF0E9EB602D0FD
:1070B000E82EFCD7F6EC35F012000501256B266BA7
:1070C000276B286B899A400EC76E200EC66E9E965F
:1070D000C69E030EC96EFF0E9EB602D0E82EFCD7E8
:1070E0009E96C69E27C5C9FFFF0E9EB602D0E82E0B
:1070F000FCD79E96C69E26C5C9FFFF0E9EB602D03F
:10710000E82EFCD79E96C69E25C5C9FFFF0E9EB6EB
:1071100002D0E82EFCD79E96C69EC952FF0E9EB6A0
:1071200002D0E82EFCD7898A0F01C950FF0A01E17D
:10713000120005012E51130A05E005012E51170A10
:107140000CE012000501E00E256FFF0E266F0F0EFA
:10715000276F000E286FB6EF38F00501E00E256F9F
:10716000FF0E266FFF0E276F000E286F899A400EC4
:10717000C76E200EC66E9E96C69E030EC96EFF0E8B
:107180009EB602D0E82EFCD79E96C69E27C5C9FFA4
:10719000FF0E9EB602D0E82EFCD79E96C69E26C550
:1071A000C9FFFF0E9EB602D0E82EFCD79E96C69E63
:1071B00025C5C9FFFF0E9EB602D0E82EFCD79E96CD
:1071C000C69EC952FF0E9EB602D0E82EFCD7898A11
:1071D0000F01C950FF0A1DE005012E51130A05E0F9
:1071E00005012E51170A0BE012000501000E256F54
:1071F000000E266F100E276F000E286F120005017B
:10720000000E256F000E266F000E276F010E286FEF
:1072100012000501256B266B276B286B05012E518B
:10722000130A05E005012E51170A0CE012000501B2
:10723000000E216F000E226F080E236F000E246FC8
:107240002BEF39F00501000E216F000E226F800E2A
:10725000236F000E246F21C500F122C501F123C563
:1072600002F124C503F125C504F126C505F127C5A2
:1072700006F128C507F1CEEC31F000C125F501C1BA
:1072800026F502C127F503C128F5899A400EC76E7D
:10729000200EC66E9E96C69E030EC96EFF0E9EB64B
:1072A00002D0E82EFCD79E96C69E27C5C9FFFF0ECA
:1072B0009EB602D0E82EFCD79E96C69E26C5C9FF74
:1072C000FF0E9EB602D0E82EFCD79E96C69E25C520
:1072D000C9FFFF0E9EB602D0E82EFCD79E96C69E32
:1072E000C952FF0E9EB602D0E82EFCD7898AC9503B
:1072F000FF0A08E104C125F505C126F506C127F5F9
:1073000007C128F5D89005012433233322332133D4
:107310002151E00B216F216795EF39F0226795EF3E
:1073200039F0236795EF39F024672BEF39F0050129
:10733000200E2527E86A2623E86A2723E86A2823FF
:107340001200E86A05012E51130A06E005012E51CC
:10735000170A0BE0020E120005012851000A03E192
:107360002751F00B07E0010E120005012851000A19
:1073700001E0010E120029C500F12AC501F12BC55B
:1073800002F12CC503F125C504F126C505F127C579
:1073900006F128C507F15DEC33F003BF1200A1EC44
:1073A00039F0D8A433EF3AF0899A400EC76E200E18
:1073B000C66E9E96C69E060EC96EFF0E9EB602D083
:1073C000E82EFCD7898A899A9E96C69E020EC96EBF
:1073D000FF0E9EB602D0E82EFCD79E96C69E27C50D
:1073E000C9FFFF0E9EB602D0E82EFCD79E96C69E21
:1073F00026C5C9FFFF0E9EB602D0E82EFCD79E968A
:10740000C69E25C5C9FFFF0E9EB602D0E82EFCD74A
:107410009E96C69E000EC96EFF0E9EB602D0E82E46
:10742000FCD7898A899A9E96C69E050EC96EFF0E64
:107430009EB602D0E82EFCD79E96C69EC952FF0E7D
:107440009EB602D0E82EFCD7C9B01CEF3AF0898A6C
:107450000501200E2527E86A2623E86A2723E86A23
:107460002823BBEF39F01200899A400EC76E200E18
:10747000C66E9E96C69E060EC96EFF0E9EB602D0C2
:10748000E82EFCD7898A899A9E96C69EC70EC96E39
:10749000FF0E9EB602D0E82EFCD7898A0501256B27
:1074A000266B276B286B1200899A400EC76E200E40
:1074B000C66E9E96C69E050EC96EFF0E9EB602D083
:1074C000E82EFCD79E96C69EC952FF0E9EB602D0ED
:1074D000E82EFCD7C9CF33F5898A1200899A400E6D
:1074E000C76E200EC66E9E96C69EB90EC96EFF0E62
:1074F0009EB602D0E82EFCD7898A1200899A400EE7
:10750000C76E200EC66E9E96C69EAB0EC96EFF0E4F
:107510009EB602D0E82EFCD7898AFF0EE82EFED751
:107520001200A1EC39F0D8A41200899A400EC76E5F
:10753000200EC66E9E96C69E030EC96EFF0E9EB6A8
:1075400002D0E82EFCD79E96C69E27C5C9FFFF0E27
:107550009EB602D0E82EFCD79E96C69E26C5C9FFD1
:10756000FF0E9EB602D0E82EFCD79E96C69E25C57D
:10757000C9FFFF0E9EB602D0E82EFCD79E96C69E8F
:10758000C952FF0E9EB602D0E82EFCD7898A0F01A1
:10759000C950FF0AD8A488EF3DF00501FE0E336FF5
:1075A000FFEC35F0ABC534F5ACC535F5ADC536F5FA
:1075B000AEC537F5AFC538F5B0C539F5B1C53AF543
:1075C0000784B6C166F1B7C167F1B8C168F1B9C146
:1075D00069F14BC14FF14CC150F14DC151F14EC158
:1075E00052F157C159F158C15AF18DEC27F000C141
:1075F0003BF501C13CF502C13DF503C13EF5050176
:107600005D670AEF3BF05E670AEF3BF05F670AEFEA
:107610003BF060670EEF3BF01BEF3BF05DC504F104
:107620005EC505F15FC506F160C507F15DEC33F09D
:1076300003BF88EF3DF059C13FF55AC140F5B5C5CC
:1076400041F5B6C542F5D5EC30F036C645F537C63E
:1076500046F50601406734EF3BF0416734EF3BF0FD
:10766000426734EF3BF0436738EF3BF049EF3BF0C4
:1076700058EC34F05EEC34F036C600F137C601F158
:1076800040C604F141C605F15DEC33F003AF88EF6D
:107690003DF00101036B026B1AC600F11BC601F13C
:1076A00001AF57EF3BF0FF0E026FFF0E036F0101BA
:1076B000076B066B1CC604F11DC605F105AF65EF2F
:1076C0003BF0FF0E066FFF0E076F62EC33F0010117
:1076D000076B066B1EC604F11FC605F105AF75EFFB
:1076E0003BF0FF0E066FFF0E076F62EC33F00101F7
:1076F000076B066B20C604F121C605F105AF85EFC7
:107700003BF0FF0E066FFF0E076F62EC33F0D89070
:1077100001010333023301330033D89001010333F5
:1077200002330133003300C147F501C148F50101BF
:10773000036B026B22C600F123C601F101AFA5EF76
:107740003BF0FF0E026FFF0E036F0101076B066B2C
:1077500024C604F125C605F105AFB3EF3BF0FF0EDB
:10776000066FFF0E076F62EC33F00101076B066BCB
:1077700026C604F127C605F105AFC3EF3BF0FF0EA7
:10778000066FFF0E076F62EC33F00101076B066BAB
:1077900028C604F129C605F105AFD3EF3BF0FF0E73
:1077A000066FFF0E076F62EC33F0D89001010333D0
:1077B000023301330033D890010103330233013324
:1077C000003300C149F501C14AF50101036B026BA9
:1077D0002AC600F12BC601F101AFF3EF3BF0FF0E1B
:1077E000026FFF0E036F0101076B066B2CC604F1DD
:1077F0002DC605F105AF01EF3CF0FF0E066FFF0E41
:10780000076F62EC33F00101076B066B2EC604F1C3
:107810002FC605F105AF11EF3CF0FF0E066FFF0E0E
:10782000076F62EC33F00101076B066B30C604F1A1
:1078300031C605F105AF21EF3CF0FF0E066FFF0EDC
:10784000076F62EC33F0D890010103330233013348
:107850000033D8900101033302330133003300C1F8
:107860004BF501C14CF50101036B026B02C600F13F
:1078700003C601F101AF41EF3CF0FF0E026FFF0EB6
:10788000036F0101076B066B04C604F105C605F121
:1078900005AF4FEF3CF0FF0E066FFF0E076F62EC77
:1078A00033F00101076B066B06C604F107C605F14C
:1078B00005AF5FEF3CF0FF0E066FFF0E076F62EC47
:1078C00033F00101076B066B08C604F109C605F128
:1078D00005AF6FEF3CF0FF0E066FFF0E076F62EC17
:1078E00033F0D89001010333023301330033D890D1
:1078F0000101033302330133003300C14DF501C1EF
:107900004EF50101036B026B0AC600F10BC601F1D3
:1079100001AF8FEF3CF0FF0E026FFF0E036F01010E
:10792000076B066B0CC604F10DC605F105AF9DEFA4
:107930003CF0FF0E066FFF0E076F62EC33F00101A3
:10794000076B066B0EC604F10FC605F105AFADEF70
:107950003CF0FF0E066FFF0E076F62EC33F0010183
:10796000076B066B10C604F111C605F105AFBDEF3C
:107970003CF0FF0E066FFF0E076F62EC33F0D890FD
:1079800001010333023301330033D8900101033383
:1079900002330133003300C14FF501C150F501013D
:1079A000036B026B12C600F113C601F101AFDDEFEC
:1079B0003CF0FF0E026FFF0E036F0101076B066BB9
:1079C00014C604F115C605F105AFEBEF3CF0FF0E50
:1079D000066FFF0E076F62EC33F00101076B066B59
:1079E00016C604F117C605F105AFFBEF3CF0FF0E1C
:1079F000066FFF0E076F62EC33F00101076B066B39
:107A000018C604F119C605F105AF0BEF3DF0FF0EE6
:107A1000066FFF0E076F62EC33F0D890010103335D
:107A2000023301330033D8900101033302330133B1
:107A3000003300C151F501C152F507940501210E33
:107A4000326F899A400EC76E200EC66E9E96C69EF5
:107A5000060EC96EFF0E9EB602D0E82EFCD7898AAC
:107A6000899A9E96C69E020EC96EFF0E9EB602D0E1
:107A7000E82EFCD79E96C69E27C5C9FFFF0E9EB670
:107A800002D0E82EFCD79E96C69E26C5C9FFFF0EE3
:107A90009EB602D0E82EFCD79E96C69E25C5C9FF8D
:107AA000FF0E9EB602D0E82EFCD725EE33F0322F23
:107AB00002D066EF3DF09E96C69EDECFC9FFFF0E58
:107AC0009EB602D0E82EFCD757EF3DF0898A899AFE
:107AD0009E96C69E050EC96EFF0E9EB602D0E82E7B
:107AE000FCD79E96C69EC952FF0E9EB602D0E82EC7
:107AF000FCD7C9B071EF3DF0898A0501200E25271A
:107B0000E86A2623E86A2723E86A282349EC32F04A
:107B1000120021C500F122C501F123C502F124C5DF
:107B200003F1899A400EC76E200EC66E9E96C69EC1
:107B30000B0EC96EFF0E9EB602D0E82EFCD79E96A5
:107B4000C69E02C1C9FFFF0E9EB602D0E82EFCD72A
:107B50009E96C69E01C1C9FFFF0E9EB602D0E82EBA
:107B6000FCD79E96C69E00C1C9FFFF0E9EB602D0EE
:107B7000E82EFCD79E96C69EC952FF0E9EB602D036
:107B8000E82EFCD725EE33F00501200E326F9E96CD
:107B9000C69EC952FF0E9EB602D0E82EFCD7C9CFB2
:107BA000DEFF322FC7EF3DF0898A1200899A400E1E
:107BB000C76E200EC66E9E96C69E900EC96EFF0EB4
:107BC0009EB602D0E82EFCD79E96C69E000EC96EC9
:107BD000FF0E9EB602D0E82EFCD79E96C69E000EE3
:107BE000C96EFF0E9EB602D0E82EFCD79E96C69EAA
:107BF000000EC96EFF0E9EB602D0E82EFCD79E96F0
:107C0000C69EC952FF0E9EB602D0E82EFCD7C9CF41
:107C10002DF59E96C69EC952FF0E9EB602D0E82E46
:107C2000FCD7C9CF2EF5898A120049EC32F0B5C5D0
:107C3000E8FFD70802E349EC32F0B5C5E8FFC80811
:107C400002E349EC32F0B5C5E8FFB90802E349ECBC
:107C500032F0B5C5E8FFAA0802E349EC32F0B5C539
:107C6000E8FF9B0802E349EC32F0A7EC36F06EEC3B
:107C70003AF0F29CF29E8B94C69AC290898C9482C0
:107C8000948C720ED36ED3A4FED789968A9093906B
:107C9000FF0EE8CF00F0E82EFED7002EFCD7815073
:107CA000F294F29A9E909D909E929D92F298F292FA
:0A7CB000F290F286F28E0300FF004E
:10BF0000E844F926000C160C2B0C3F0C520C640C68
:10BF1000760C860C960CA50CB30CC10CCF0CDC0C6B
:06BF2000E80CF40C000C1B
:00000001FF
